BL51 BANKED LINKER/LOCATER V6.22                                                        12/05/2013  00:54:40  PAGE 1


BL51 BANKED LINKER/LOCATER V6.22, INVOKED BY:
C:\KEIL4\C51\BIN\BL51.EXE ..\OBJ\main.obj, ..\OBJ\LCD drive.obj, ..\OBJ\Touch.obj TO ..\OBJ\LCD PRINT (.\LCD.m51) RAMSIZ
>> E (256)


MEMORY MODEL: SMALL WITH FLOATING POINT ARITHMETIC


INPUT MODULES INCLUDED:
  ..\OBJ\main.obj (MAIN)
  ..\OBJ\LCD drive.obj (LCD_DRIVE)
  ..\OBJ\Touch.obj (TOUCH)
  C:\KEIL4\C51\LIB\C51FPS.LIB (?C?FPMUL)
  C:\KEIL4\C51\LIB\C51FPS.LIB (?C?FPDIV)
  C:\KEIL4\C51\LIB\C51FPS.LIB (?C?FCAST)
  C:\KEIL4\C51\LIB\C51FPS.LIB (?C?CASTF)
  C:\KEIL4\C51\LIB\C51FPS.LIB (?C?FPGETOPN)
  C:\KEIL4\C51\LIB\C51S.LIB (?C_STARTUP)
  C:\KEIL4\C51\LIB\C51S.LIB (?C?COPY)
  C:\KEIL4\C51\LIB\C51S.LIB (?C?LNEG)


LINK MAP OF MODULE:  ..\OBJ\LCD (MAIN)


            TYPE    BASE      LENGTH    RELOCATION   SEGMENT NAME
            -----------------------------------------------------

            * * * * * * *   D A T A   M E M O R Y   * * * * * * *
            REG     0000H     0008H     ABSOLUTE     "REG BANK 0"
            DATA    0008H     001CH     UNIT         _DATA_GROUP_
            DATA    0024H     0008H     UNIT         ?DT?TOUCH
            DATA    002CH     0006H     UNIT         ?DT?MAIN
            IDATA   0032H     0001H     UNIT         ?STACK

            * * * * * * *   C O D E   M E M O R Y   * * * * * * *
            CODE    0000H     0003H     ABSOLUTE     
            CODE    0003H     2875H     UNIT         ?PR?LCD_INIT?LCD_DRIVE
            CODE    2878H     06C3H     UNIT         ?CO?LCD_DRIVE
            CODE    2F3BH     0369H     UNIT         ?C?LIB_CODE
            CODE    32A4H     0348H     UNIT         ?PR?DISPLAY_ID?LCD_DRIVE
            CODE    35ECH     027FH     UNIT         ?PR?_LCD_TEST_SINGLECOLOR?LCD_DRIVE
            CODE    386BH     01B4H     UNIT         ?PR?_LCD_SETPOS?TOUCH
            CODE    3A1FH     0164H     UNIT         ?PR?_LCD_SETWINDOW?LCD_DRIVE
            CODE    3B83H     00E8H     UNIT         ?PR?MAIN?MAIN
            CODE    3C6BH     00C7H     UNIT         ?PR?_LCD_ID_61581?LCD_DRIVE
            CODE    3D32H     00C7H     UNIT         ?PR?GETPIX?TOUCH
            CODE    3DF9H     00C4H     UNIT         ?PR?_GUI_SPRINTF_CHAR?LCD_DRIVE
            CODE    3EBDH     0094H     UNIT         ?PR?_LCD_ID?LCD_DRIVE
            CODE    3F51H     0083H     UNIT         ?PR?PIX_FILTER?TOUCH
            CODE    3FD4H     0081H     UNIT         ?PR?_LCD_ID_9341?LCD_DRIVE
            CODE    4055H     004FH     UNIT         ?PR?_GUI_SPRINTF_STRING?LCD_DRIVE
            CODE    40A4H     0047H     UNIT         ?PR?_LCD_WRITE_DATA?LCD_DRIVE
            CODE    40EBH     0041H     UNIT         ?PR?_DRAWPOINT?TOUCH
            CODE    412CH     0040H     UNIT         ?PR?_DELAYMS?LCD_DRIVE
            CODE    416CH     0039H     UNIT         ?PR?_LLCD_WRITE_CMD?LCD_DRIVE
            CODE    41A5H     0038H     UNIT         ?PR?_LLCD_WRITE_DATA?LCD_DRIVE
            CODE    41DDH     002DH     UNIT         ?PR?_LCD_WRITE_CMD?LCD_DRIVE
BL51 BANKED LINKER/LOCATER V6.22                                                      12/05/2013  00:54:40  PAGE 2


            CODE    420AH     002AH     UNIT         ?PR?LCD_READ_8347ID?LCD_DRIVE
            CODE    4234H     0029H     UNIT         ?PR?_UART_SEND_DATA?LCD_DRIVE
            CODE    425DH     0029H     UNIT         ?PR?LCD_READ_ID?LCD_DRIVE
            CODE    4286H     0026H     UNIT         ?PR?LCD_READ_ID9341?LCD_DRIVE
            CODE    42ACH     0023H     UNIT         ?PR?AD7843?TOUCH
            CODE    42CFH     001FH     UNIT         ?PR?LCD_READ_ID61581?LCD_DRIVE
            CODE    42EEH     001FH     UNIT         ?PR?_WRITE_7843?TOUCH
            CODE    430DH     001FH     UNIT         ?PR?READ_7843?TOUCH
            CODE    432CH     001DH     UNIT         ?PR?_DELAY?TOUCH
            CODE    4349H     001AH     UNIT         ?PR?HD_RESET?LCD_DRIVE
            CODE    4363H     0016H     UNIT         ?PR?_SENG_CMD_DAT?LCD_DRIVE
            CODE    4379H     000FH     UNIT         ?PR?UART_INIT?LCD_DRIVE
            CODE    4388H     000EH     UNIT         ?PR?_GUI_POINT?LCD_DRIVE
            CODE    4396H     000DH     UNIT         ?PR?KEYPRESS?LCD_DRIVE
            CODE    43A3H     000CH     UNIT         ?PR?_DELAYUS?LCD_DRIVE
            CODE    43AFH     000CH     UNIT         ?C_C51STARTUP
            CODE    43BBH     000BH     UNIT         ?PR?START_7843?TOUCH
            CODE    43C6H     0009H     UNIT         ?PR?_LCD_SETXY?LCD_DRIVE



OVERLAY MAP OF MODULE:   ..\OBJ\LCD (MAIN)


SEGMENT                                       DATA_GROUP 
  +--> CALLED SEGMENT                       START    LENGTH
-----------------------------------------------------------
?C_C51STARTUP                               -----    -----
  +--> ?PR?MAIN?MAIN

?PR?MAIN?MAIN                               -----    -----
  +--> ?PR?LCD_READ_ID9341?LCD_DRIVE
  +--> ?PR?LCD_READ_ID61581?LCD_DRIVE
  +--> ?PR?LCD_READ_ID?LCD_DRIVE
  +--> ?PR?LCD_READ_8347ID?LCD_DRIVE
  +--> ?PR?LCD_INIT?LCD_DRIVE
  +--> ?PR?KEYPRESS?LCD_DRIVE
  +--> ?PR?_LCD_TEST_SINGLECOLOR?LCD_DRIVE
  +--> ?PR?DISPLAY_ID?LCD_DRIVE
  +--> ?PR?GETPIX?TOUCH
  +--> ?PR?_DRAWPOINT?TOUCH

?PR?LCD_READ_ID9341?LCD_DRIVE               -----    -----
  +--> ?PR?HD_RESET?LCD_DRIVE
  +--> ?PR?_DELAYMS?LCD_DRIVE
  +--> ?PR?_LCD_ID_9341?LCD_DRIVE
  +--> ?PR?_UART_SEND_DATA?LCD_DRIVE

?PR?HD_RESET?LCD_DRIVE                      -----    -----
  +--> ?PR?UART_INIT?LCD_DRIVE
  +--> ?PR?_DELAYMS?LCD_DRIVE

?PR?_DELAYMS?LCD_DRIVE                      0010H    0002H
  +--> ?PR?_UART_SEND_DATA?LCD_DRIVE
  +--> ?PR?_DELAYUS?LCD_DRIVE

?PR?_UART_SEND_DATA?LCD_DRIVE               -----    -----
BL51 BANKED LINKER/LOCATER V6.22                                                      12/05/2013  00:54:40  PAGE 3


  +--> ?PR?UART_INIT?LCD_DRIVE

?PR?_LCD_ID_9341?LCD_DRIVE                  0008H    0006H
  +--> ?PR?_LLCD_WRITE_CMD?LCD_DRIVE
  +--> ?PR?_DELAYMS?LCD_DRIVE
  +--> ?PR?_UART_SEND_DATA?LCD_DRIVE

?PR?LCD_READ_ID61581?LCD_DRIVE              -----    -----
  +--> ?PR?HD_RESET?LCD_DRIVE
  +--> ?PR?_DELAYMS?LCD_DRIVE
  +--> ?PR?_LCD_ID_61581?LCD_DRIVE
  +--> ?PR?_UART_SEND_DATA?LCD_DRIVE

?PR?_LCD_ID_61581?LCD_DRIVE                 0008H    0004H
  +--> ?PR?_LLCD_WRITE_CMD?LCD_DRIVE
  +--> ?PR?_LLCD_WRITE_DATA?LCD_DRIVE
  +--> ?PR?_DELAYMS?LCD_DRIVE
  +--> ?PR?_UART_SEND_DATA?LCD_DRIVE

?PR?LCD_READ_ID?LCD_DRIVE                   -----    -----
  +--> ?PR?HD_RESET?LCD_DRIVE
  +--> ?PR?_DELAYMS?LCD_DRIVE
  +--> ?PR?_SENG_CMD_DAT?LCD_DRIVE
  +--> ?PR?_LCD_ID?LCD_DRIVE
  +--> ?PR?_UART_SEND_DATA?LCD_DRIVE

?PR?_SENG_CMD_DAT?LCD_DRIVE                 -----    -----
  +--> ?PR?_LLCD_WRITE_CMD?LCD_DRIVE
  +--> ?PR?_LLCD_WRITE_DATA?LCD_DRIVE

?PR?_LCD_ID?LCD_DRIVE                       0008H    0008H
  +--> ?PR?_LLCD_WRITE_CMD?LCD_DRIVE
  +--> ?PR?_DELAYMS?LCD_DRIVE

?PR?LCD_READ_8347ID?LCD_DRIVE               -----    -----
  +--> ?PR?HD_RESET?LCD_DRIVE
  +--> ?PR?_DELAYMS?LCD_DRIVE
  +--> ?PR?_SENG_CMD_DAT?LCD_DRIVE
  +--> ?PR?_LCD_ID?LCD_DRIVE
  +--> ?PR?_UART_SEND_DATA?LCD_DRIVE

?PR?LCD_INIT?LCD_DRIVE                      -----    -----
  +--> ?PR?_DELAYMS?LCD_DRIVE
  +--> ?PR?_SENG_CMD_DAT?LCD_DRIVE
  +--> ?PR?_LLCD_WRITE_CMD?LCD_DRIVE
  +--> ?PR?_LLCD_WRITE_DATA?LCD_DRIVE
  +--> ?PR?_LCD_TEST_SINGLECOLOR?LCD_DRIVE

?PR?_LCD_TEST_SINGLECOLOR?LCD_DRIVE         0008H    0003H
  +--> ?PR?_LCD_WRITE_DATA?LCD_DRIVE
  +--> ?PR?_LCD_WRITE_CMD?LCD_DRIVE
  +--> ?PR?_LLCD_WRITE_CMD?LCD_DRIVE
  +--> ?PR?_SENG_CMD_DAT?LCD_DRIVE
  +--> ?PR?_LLCD_WRITE_DATA?LCD_DRIVE

?PR?_LCD_WRITE_DATA?LCD_DRIVE               -----    -----
  +--> ?PR?_LCD_WRITE_CMD?LCD_DRIVE
BL51 BANKED LINKER/LOCATER V6.22                                                      12/05/2013  00:54:40  PAGE 4



?PR?KEYPRESS?LCD_DRIVE                      -----    -----
  +--> ?PR?_DELAYMS?LCD_DRIVE

?PR?DISPLAY_ID?LCD_DRIVE                    -----    -----
  +--> ?CO?LCD_DRIVE
  +--> ?PR?_GUI_SPRINTF_STRING?LCD_DRIVE

?PR?_GUI_SPRINTF_STRING?LCD_DRIVE           0008H    0009H
  +--> ?CO?LCD_DRIVE
  +--> ?PR?_GUI_SPRINTF_CHAR?LCD_DRIVE

?PR?_GUI_SPRINTF_CHAR?LCD_DRIVE             0011H    000BH
  +--> ?CO?LCD_DRIVE
  +--> ?PR?_GUI_POINT?LCD_DRIVE

?PR?_GUI_POINT?LCD_DRIVE                    001CH    0002H
  +--> ?PR?_LCD_SETXY?LCD_DRIVE
  +--> ?PR?_LLCD_WRITE_DATA?LCD_DRIVE

?PR?_LCD_SETXY?LCD_DRIVE                    -----    -----
  +--> ?PR?_LCD_SETWINDOW?LCD_DRIVE

?PR?_LCD_SETWINDOW?LCD_DRIVE                001EH    0006H
  +--> ?PR?_SENG_CMD_DAT?LCD_DRIVE
  +--> ?PR?_LLCD_WRITE_CMD?LCD_DRIVE
  +--> ?PR?_LLCD_WRITE_DATA?LCD_DRIVE

?PR?GETPIX?TOUCH                            0008H    0009H
  +--> ?PR?AD7843?TOUCH
  +--> ?PR?PIX_FILTER?TOUCH

?PR?AD7843?TOUCH                            0011H    0004H
  +--> ?PR?_DELAY?TOUCH
  +--> ?PR?READ_7843?TOUCH

?PR?_DELAY?TOUCH                            -----    -----
  +--> ?PR?_WRITE_7843?TOUCH

?PR?READ_7843?TOUCH                         -----    -----
  +--> ?PR?_DELAY?TOUCH

?PR?PIX_FILTER?TOUCH                        0011H    0008H

?PR?_DRAWPOINT?TOUCH                        0008H    0002H
  +--> ?PR?_LCD_SETPOS?TOUCH
  +--> ?PR?_LLCD_WRITE_DATA?LCD_DRIVE

?PR?_LCD_SETPOS?TOUCH                       000AH    0008H
  +--> ?PR?_SENG_CMD_DAT?LCD_DRIVE
  +--> ?PR?_LLCD_WRITE_CMD?LCD_DRIVE
  +--> ?PR?_LLCD_WRITE_DATA?LCD_DRIVE



SYMBOL TABLE OF MODULE:  ..\OBJ\LCD (MAIN)

BL51 BANKED LINKER/LOCATER V6.22                                                      12/05/2013  00:54:40  PAGE 5


  VALUE           TYPE          NAME
  ----------------------------------

  -------         MODULE        MAIN
  C:0000H         SYMBOL        _ICE_DUMMY_
  D:0090H         PUBLIC        P1
  D:00B0H         PUBLIC        P3
  D:002CH         PUBLIC        tempid
  D:00A8H         PUBLIC        IE
  D:00B8H         PUBLIC        IP
  C:3B83H         PUBLIC        main
  D:002EH         PUBLIC        zhiyi
  D:0098H         PUBLIC        SCON
  D:0088H         PUBLIC        TCON
  D:0030H         PUBLIC        temp
  D:00C8H         PUBLIC        T2CON
  D:00D0H         PUBLIC        PSW
  -------         PROC          MAIN
  -------         DO            
  D:0007H         SYMBOL        bawei
  -------         ENDDO         
  C:3B83H         LINE#         10
  C:3B83H         LINE#         11
  C:3B83H         LINE#         14
  C:3B88H         LINE#         18
  C:3B8BH         LINE#         19
  C:3B91H         LINE#         20
  C:3B91H         LINE#         21
  C:3B94H         LINE#         22
  C:3B94H         LINE#         25
  C:3BACH         LINE#         26
  C:3BACH         LINE#         27
  C:3BAFH         LINE#         28
  C:3BAFH         LINE#         31
  C:3BB5H         LINE#         32
  C:3BB5H         LINE#         33
  C:3BB8H         LINE#         34
  C:3BC0H         LINE#         35
  C:3BC0H         LINE#         36
  C:3BC6H         LINE#         37
  C:3BC6H         LINE#         38
  C:3BC6H         LINE#         39
  C:3BC8H         LINE#         41
  C:3BCBH         LINE#         42
  C:3BCBH         LINE#         43
  C:3BD1H         LINE#         44
  C:3BD4H         LINE#         45
  C:3BD4H         LINE#         50
  C:3BD7H         LINE#         52
  C:3BD7H         LINE#         53
  C:3BD7H         LINE#         55
  C:3BE3H         LINE#         56
  C:3BE3H         LINE#         58
  C:3BEFH         LINE#         59
  C:3BEFH         LINE#         60
  C:3BF2H         LINE#         61
  C:3BF2H         LINE#         69
BL51 BANKED LINKER/LOCATER V6.22                                                      12/05/2013  00:54:40  PAGE 6


  C:3BF2H         LINE#         71
  C:3BFAH         LINE#         72
  C:3BFAH         LINE#         74
  C:3C06H         LINE#         75
  C:3C06H         LINE#         76
  C:3C09H         LINE#         77
  C:3C09H         LINE#         82
  C:3C0FH         LINE#         83
  C:3C12H         LINE#         84
  C:3C12H         LINE#         85
  C:3C19H         LINE#         87
  C:3C25H         LINE#         88
  C:3C25H         LINE#         89
  C:3C28H         LINE#         90
  C:3C28H         LINE#         98
  C:3C2FH         LINE#         100
  C:3C3BH         LINE#         101
  C:3C3BH         LINE#         102
  C:3C3EH         LINE#         103
  C:3C3EH         LINE#         111
  C:3C44H         LINE#         114
  C:3C50H         LINE#         115
  C:3C50H         LINE#         116
  C:3C53H         LINE#         117
  C:3C53H         LINE#         122
  C:3C56H         LINE#         126
  C:3C56H         LINE#         127
  C:3C56H         LINE#         128
  C:3C5CH         LINE#         129
  C:3C5CH         LINE#         130
  C:3C69H         LINE#         131
  C:3C69H         LINE#         132
  -------         ENDPROC       MAIN
  -------         ENDMOD        MAIN

  -------         MODULE        LCD_DRIVE
  C:0000H         SYMBOL        _ICE_DUMMY_
  D:0080H         PUBLIC        P0
  C:425DH         PUBLIC        LCD_read_id
  D:0090H         PUBLIC        P1
  D:00A0H         PUBLIC        P2
  D:00B0H         PUBLIC        P3
  C:42CFH         PUBLIC        LCD_read_id61581
  C:41A8H         PUBLIC        _LLCD_WRITE_DATA
  D:00A8H         PUBLIC        IE
  C:4351H         PUBLIC        HD_reset
  D:00B8H         PUBLIC        IP
  B:0098H.1       PUBLIC        TI
  C:3A1FH         PUBLIC        _LCD_setwindow
  B:0090H.1       PUBLIC        RS
  C:3C6BH         PUBLIC        _LCD_ID_61581
  D:0099H         PUBLIC        SBUF
  D:0098H         PUBLIC        SCON
  D:0089H         PUBLIC        TMOD
  D:0088H         PUBLIC        TCON
  C:40BEH         PUBLIC        _LCD_WRITE_DATA
  C:35ECH         PUBLIC        _LCD_TEST_SingleColor
BL51 BANKED LINKER/LOCATER V6.22                                                      12/05/2013  00:54:40  PAGE 7


  C:3EBDH         PUBLIC        _LCD_ID
  C:4170H         PUBLIC        _LLCD_WRITE_CMD
  C:4255H         PUBLIC        _UART_send_data
  C:32A4H         PUBLIC        Display_ID
  C:4069H         PUBLIC        _GUI_sprintf_string
  D:008DH         PUBLIC        TH1
  D:008BH         PUBLIC        TL1
  C:294BH         PUBLIC        font16x8
  C:3DF9H         PUBLIC        _GUI_sprintf_char
  C:4388H         PUBLIC        _GUI_Point
  C:4286H         PUBLIC        LCD_read_id9341
  C:4379H         PUBLIC        UART_init
  B:0088H.6       PUBLIC        TR1
  C:420AH         PUBLIC        LCD_read_8347id
  B:0090H.3       PUBLIC        RDB
  C:4396H         PUBLIC        Keypress
  C:436BH         PUBLIC        _seng_cmd_dat
  B:0090H.0       PUBLIC        TFT_CS
  D:00C8H         PUBLIC        T2CON
  B:00B0H.3       PUBLIC        KEY
  C:0003H         PUBLIC        LCD_init
  B:0090H.4       PUBLIC        RES
  B:0090H.2       PUBLIC        WRB
  C:4150H         PUBLIC        _delayms
  C:3FD4H         PUBLIC        _LCD_ID_9341
  C:43C6H         PUBLIC        _LCD_setxy
  C:41DDH         PUBLIC        _LCD_WRITE_CMD
  D:00D0H         PUBLIC        PSW
  C:43A3H         PUBLIC        _delayus
  -------         PROC          UART_INIT
  C:4379H         LINE#         8
  C:4379H         LINE#         9
  C:4379H         LINE#         10
  C:437CH         LINE#         11
  C:437FH         LINE#         12
  C:4382H         LINE#         13
  C:4385H         LINE#         14
  C:4387H         LINE#         16
  -------         ENDPROC       UART_INIT
  C:423DH         SYMBOL        L?0376
  -------         PROC          L?0375
  -------         ENDPROC       L?0375
  C:423DH         SYMBOL        L?0376
  -------         PROC          _UART_SEND_DATA
  D:0007H         SYMBOL        lcdid
  C:4255H         LINE#         21
  C:4255H         LINE#         22
  C:4255H         LINE#         24
  C:4257H         LINE#         25
  C:425AH         LINE#         26
  C:425CH         LINE#         28
  -------         ENDPROC       _UART_SEND_DATA
  -------         PROC          DISPLAY_ID
  C:32A4H         LINE#         34
  C:32A4H         LINE#         35
  C:32A4H         LINE#         36
  C:32B0H         LINE#         37
BL51 BANKED LINKER/LOCATER V6.22                                                      12/05/2013  00:54:40  PAGE 8


  C:32B0H         LINE#         38
  C:32B7H         LINE#         39
  C:32BFH         LINE#         40
  C:32BFH         LINE#         41
  C:32C3H         LINE#         42
  C:32C6H         LINE#         43
  C:32C6H         LINE#         44
  C:32CAH         LINE#         45
  C:32CAH         LINE#         46
  C:32D9H         LINE#         47
  C:32D9H         LINE#         48
  C:32E0H         LINE#         49
  C:32E8H         LINE#         50
  C:32E8H         LINE#         51
  C:32ECH         LINE#         52
  C:32EEH         LINE#         53
  C:32EEH         LINE#         54
  C:32F2H         LINE#         55
  C:32F2H         LINE#         56
  C:32F5H         LINE#         57
  C:3301H         LINE#         58
  C:3301H         LINE#         59
  C:3304H         LINE#         60
  C:330CH         LINE#         61
  C:330CH         LINE#         62
  C:3310H         LINE#         63
  C:3312H         LINE#         64
  C:3312H         LINE#         65
  C:3316H         LINE#         66
  C:3316H         LINE#         67
  C:3319H         LINE#         68
  C:3325H         LINE#         69
  C:3325H         LINE#         70
  C:3328H         LINE#         71
  C:3330H         LINE#         72
  C:3330H         LINE#         73
  C:3334H         LINE#         74
  C:3336H         LINE#         75
  C:3336H         LINE#         76
  C:333AH         LINE#         77
  C:333AH         LINE#         78
  C:3349H         LINE#         79
  C:3349H         LINE#         80
  C:3350H         LINE#         81
  C:3358H         LINE#         82
  C:3358H         LINE#         83
  C:335CH         LINE#         84
  C:335EH         LINE#         85
  C:335EH         LINE#         86
  C:3362H         LINE#         87
  C:3362H         LINE#         88
  C:3365H         LINE#         89
  C:3371H         LINE#         90
  C:3371H         LINE#         91
  C:3378H         LINE#         92
  C:3380H         LINE#         93
  C:3380H         LINE#         94
BL51 BANKED LINKER/LOCATER V6.22                                                      12/05/2013  00:54:40  PAGE 9


  C:3384H         LINE#         95
  C:3386H         LINE#         96
  C:3386H         LINE#         97
  C:338AH         LINE#         98
  C:338AH         LINE#         99
  C:3399H         LINE#         100
  C:3399H         LINE#         101
  C:33A0H         LINE#         102
  C:33A8H         LINE#         103
  C:33A8H         LINE#         104
  C:33ACH         LINE#         105
  C:33AEH         LINE#         106
  C:33AEH         LINE#         107
  C:33B2H         LINE#         108
  C:33B2H         LINE#         109
  C:33B5H         LINE#         110
  C:33C1H         LINE#         111
  C:33C1H         LINE#         112
  C:33C8H         LINE#         113
  C:33D0H         LINE#         114
  C:33D0H         LINE#         115
  C:33D4H         LINE#         116
  C:33D6H         LINE#         117
  C:33D6H         LINE#         118
  C:33DAH         LINE#         119
  C:33DAH         LINE#         120
  C:33DDH         LINE#         121
  C:33E9H         LINE#         122
  C:33E9H         LINE#         123
  C:33F0H         LINE#         124
  C:33F8H         LINE#         125
  C:33F8H         LINE#         126
  C:33FCH         LINE#         127
  C:33FEH         LINE#         128
  C:33FEH         LINE#         129
  C:3402H         LINE#         130
  C:3402H         LINE#         131
  C:3405H         LINE#         132
  C:3411H         LINE#         133
  C:3411H         LINE#         134
  C:3418H         LINE#         135
  C:3420H         LINE#         136
  C:3420H         LINE#         137
  C:3424H         LINE#         138
  C:3426H         LINE#         139
  C:3426H         LINE#         140
  C:342AH         LINE#         141
  C:342AH         LINE#         142
  C:3439H         LINE#         143
  C:3439H         LINE#         144
  C:3440H         LINE#         145
  C:3448H         LINE#         146
  C:3448H         LINE#         147
  C:344CH         LINE#         148
  C:344EH         LINE#         149
  C:344EH         LINE#         150
  C:3452H         LINE#         151
BL51 BANKED LINKER/LOCATER V6.22                                                      12/05/2013  00:54:40  PAGE 10


  C:3452H         LINE#         152
  C:3455H         LINE#         153
  C:3461H         LINE#         154
  C:3461H         LINE#         155
  C:3468H         LINE#         156
  C:3470H         LINE#         157
  C:3470H         LINE#         158
  C:3474H         LINE#         159
  C:3476H         LINE#         160
  C:3476H         LINE#         161
  C:347AH         LINE#         162
  C:347AH         LINE#         163
  C:3489H         LINE#         164
  C:3489H         LINE#         165
  C:3490H         LINE#         166
  C:3498H         LINE#         167
  C:3498H         LINE#         168
  C:349CH         LINE#         169
  C:349EH         LINE#         170
  C:349EH         LINE#         171
  C:34A2H         LINE#         172
  C:34A2H         LINE#         173
  C:34B1H         LINE#         174
  C:34B1H         LINE#         175
  C:34B8H         LINE#         176
  C:34C0H         LINE#         177
  C:34C0H         LINE#         178
  C:34C4H         LINE#         179
  C:34C6H         LINE#         180
  C:34C6H         LINE#         181
  C:34CAH         LINE#         182
  C:34CAH         LINE#         183
  C:34D9H         LINE#         184
  C:34D9H         LINE#         185
  C:34E0H         LINE#         186
  C:34E8H         LINE#         187
  C:34E8H         LINE#         188
  C:34ECH         LINE#         189
  C:34EEH         LINE#         190
  C:34EEH         LINE#         191
  C:34F2H         LINE#         192
  C:34F2H         LINE#         193
  C:3501H         LINE#         194
  C:3501H         LINE#         195
  C:3508H         LINE#         196
  C:3510H         LINE#         197
  C:3510H         LINE#         198
  C:3514H         LINE#         199
  C:3516H         LINE#         200
  C:3516H         LINE#         201
  C:351AH         LINE#         202
  C:351AH         LINE#         203
  C:3529H         LINE#         204
  C:3529H         LINE#         205
  C:3530H         LINE#         206
  C:3538H         LINE#         207
  C:3538H         LINE#         208
BL51 BANKED LINKER/LOCATER V6.22                                                      12/05/2013  00:54:40  PAGE 11


  C:353CH         LINE#         209
  C:353EH         LINE#         210
  C:353EH         LINE#         211
  C:3542H         LINE#         212
  C:3542H         LINE#         213
  C:3551H         LINE#         214
  C:3551H         LINE#         215
  C:3558H         LINE#         216
  C:3560H         LINE#         217
  C:3560H         LINE#         218
  C:3564H         LINE#         219
  C:3566H         LINE#         220
  C:3566H         LINE#         221
  C:356AH         LINE#         222
  C:356AH         LINE#         223
  C:3579H         LINE#         224
  C:3579H         LINE#         225
  C:3580H         LINE#         226
  C:3588H         LINE#         227
  C:3588H         LINE#         228
  C:358CH         LINE#         229
  C:358EH         LINE#         230
  C:358EH         LINE#         231
  C:3592H         LINE#         232
  C:3592H         LINE#         233
  C:359CH         LINE#         234
  C:359CH         LINE#         235
  C:35A3H         LINE#         236
  C:35ABH         LINE#         237
  C:35ABH         LINE#         238
  C:35AFH         LINE#         239
  C:35B1H         LINE#         240
  C:35B1H         LINE#         241
  C:35B5H         LINE#         242
  C:35B5H         LINE#         243
  C:35BFH         LINE#         244
  C:35BFH         LINE#         245
  C:35C6H         LINE#         246
  C:35CEH         LINE#         247
  C:35CEH         LINE#         248
  C:35D2H         LINE#         249
  C:35D4H         LINE#         250
  C:35D4H         LINE#         251
  C:35EBH         LINE#         252
  C:35EBH         LINE#         253
  C:35EBH         LINE#         255
  -------         ENDPROC       DISPLAY_ID
  -------         PROC          LCD_INIT
  C:0003H         LINE#         260
  C:0003H         LINE#         261
  C:0003H         LINE#         262
  C:0012H         LINE#         263
  C:0012H         LINE#         264
  C:0018H         LINE#         265
  C:0020H         LINE#         266
  C:0028H         LINE#         267
  C:0030H         LINE#         268
BL51 BANKED LINKER/LOCATER V6.22                                                      12/05/2013  00:54:40  PAGE 12


  C:0038H         LINE#         269
  C:003FH         LINE#         270
  C:004AH         LINE#         271
  C:0054H         LINE#         273
  C:005FH         LINE#         274
  C:006AH         LINE#         275
  C:0075H         LINE#         276
  C:0080H         LINE#         277
  C:008BH         LINE#         278
  C:0096H         LINE#         279
  C:00A1H         LINE#         280
  C:00ACH         LINE#         281
  C:00B7H         LINE#         282
  C:00C2H         LINE#         284
  C:00CDH         LINE#         285
  C:00D8H         LINE#         286
  C:00E1H         LINE#         287
  C:00E6H         LINE#         289
  C:00F1H         LINE#         290
  C:00FCH         LINE#         291
  C:0107H         LINE#         292
  C:0112H         LINE#         293
  C:011DH         LINE#         294
  C:0124H         LINE#         296
  C:012FH         LINE#         297
  C:013AH         LINE#         298
  C:0145H         LINE#         299
  C:0150H         LINE#         300
  C:0159H         LINE#         301
  C:0164H         LINE#         302
  C:016DH         LINE#         304
  C:0177H         LINE#         305
  C:0182H         LINE#         306
  C:018CH         LINE#         307
  C:0197H         LINE#         308
  C:01A0H         LINE#         309
  C:01AAH         LINE#         310
  C:01B5H         LINE#         311
  C:01C0H         LINE#         312
  C:01CAH         LINE#         313
  C:01D1H         LINE#         315
  C:01DCH         LINE#         316
  C:01E3H         LINE#         318
  C:01ECH         LINE#         319
  C:01F6H         LINE#         320
  C:01FAH         LINE#         321
  C:01FAH         LINE#         324
  C:020CH         LINE#         325
  C:020CH         LINE#         381
  C:0219H         LINE#         382
  C:0227H         LINE#         383
  C:0231H         LINE#         384
  C:023FH         LINE#         385
  C:024DH         LINE#         386
  C:025BH         LINE#         387
  C:0269H         LINE#         388
  C:0270H         LINE#         389
BL51 BANKED LINKER/LOCATER V6.22                                                      12/05/2013  00:54:40  PAGE 13


  C:027AH         LINE#         390
  C:0281H         LINE#         391
  C:028BH         LINE#         392
  C:0292H         LINE#         393
  C:029CH         LINE#         394
  C:02A3H         LINE#         395
  C:02ADH         LINE#         396
  C:02B4H         LINE#         397
  C:02BEH         LINE#         398
  C:02CCH         LINE#         399
  C:02DAH         LINE#         400
  C:02E8H         LINE#         401
  C:02F6H         LINE#         402
  C:0304H         LINE#         403
  C:030EH         LINE#         404
  C:031CH         LINE#         405
  C:032AH         LINE#         407
  C:0334H         LINE#         408
  C:0342H         LINE#         409
  C:034FH         LINE#         410
  C:035DH         LINE#         411
  C:036AH         LINE#         412
  C:0378H         LINE#         413
  C:0385H         LINE#         415
  C:0393H         LINE#         416
  C:03A1H         LINE#         417
  C:03AFH         LINE#         418
  C:03BDH         LINE#         419
  C:03CBH         LINE#         420
  C:03D9H         LINE#         421
  C:03E7H         LINE#         422
  C:03F4H         LINE#         423
  C:0402H         LINE#         424
  C:0410H         LINE#         426
  C:041EH         LINE#         428
  C:0425H         LINE#         429
  C:0433H         LINE#         430
  C:043AH         LINE#         431
  C:0448H         LINE#         432
  C:044FH         LINE#         433
  C:045DH         LINE#         434
  C:045DH         LINE#         436
  C:0460H         LINE#         437
  C:046CH         LINE#         438
  C:046CH         LINE#         440
  C:046CH         LINE#         441
  C:046CH         LINE#         442
  C:046CH         LINE#         443
  C:046CH         LINE#         444
  C:046CH         LINE#         445
  C:046CH         LINE#         446
  C:046CH         LINE#         447
  C:046CH         LINE#         448
  C:046CH         LINE#         449
  C:046CH         LINE#         450
  C:046CH         LINE#         451
  C:046CH         LINE#         452
BL51 BANKED LINKER/LOCATER V6.22                                                      12/05/2013  00:54:40  PAGE 14


  C:046CH         LINE#         453
  C:046CH         LINE#         454
  C:046CH         LINE#         455
  C:046CH         LINE#         456
  C:046CH         LINE#         457
  C:046CH         LINE#         458
  C:046CH         LINE#         459
  C:046CH         LINE#         460
  C:046CH         LINE#         461
  C:046CH         LINE#         462
  C:046CH         LINE#         465
  C:046CH         LINE#         466
  C:046CH         LINE#         467
  C:046CH         LINE#         468
  C:046CH         LINE#         469
  C:046CH         LINE#         470
  C:046CH         LINE#         471
  C:046CH         LINE#         472
  C:046CH         LINE#         473
  C:046CH         LINE#         474
  C:046CH         LINE#         475
  C:046CH         LINE#         478
  C:046CH         LINE#         479
  C:046CH         LINE#         480
  C:046CH         LINE#         481
  C:046CH         LINE#         482
  C:046CH         LINE#         483
  C:046CH         LINE#         484
  C:046CH         LINE#         485
  C:046CH         LINE#         486
  C:046CH         LINE#         487
  C:046CH         LINE#         488
  C:046CH         LINE#         490
  C:046EH         LINE#         491
  C:047DH         LINE#         492
  C:047DH         LINE#         494
  C:0486H         LINE#         495
  C:0491H         LINE#         496
  C:049CH         LINE#         497
  C:04A7H         LINE#         498
  C:04B2H         LINE#         499
  C:04BDH         LINE#         500
  C:04C8H         LINE#         501
  C:04D1H         LINE#         502
  C:04DAH         LINE#         503
  C:04E3H         LINE#         504
  C:04EEH         LINE#         505
  C:04F7H         LINE#         506
  C:0500H         LINE#         507
  C:0507H         LINE#         508
  C:0512H         LINE#         509
  C:0519H         LINE#         510
  C:0524H         LINE#         511
  C:052BH         LINE#         512
  C:0536H         LINE#         513
  C:053DH         LINE#         514
  C:0548H         LINE#         515
BL51 BANKED LINKER/LOCATER V6.22                                                      12/05/2013  00:54:40  PAGE 15


  C:054FH         LINE#         516
  C:055AH         LINE#         519
  C:0563H         LINE#         520
  C:056EH         LINE#         521
  C:0579H         LINE#         522
  C:0584H         LINE#         523
  C:058FH         LINE#         524
  C:0598H         LINE#         525
  C:05A3H         LINE#         526
  C:05AEH         LINE#         527
  C:05B9H         LINE#         528
  C:05C4H         LINE#         529
  C:05CBH         LINE#         532
  C:05D4H         LINE#         533
  C:05DFH         LINE#         534
  C:05E8H         LINE#         535
  C:05F3H         LINE#         536
  C:05FEH         LINE#         537
  C:0609H         LINE#         538
  C:0614H         LINE#         539
  C:061FH         LINE#         540
  C:062AH         LINE#         541
  C:062CH         LINE#         543
  C:062CH         LINE#         545
  C:063EH         LINE#         546
  C:063EH         LINE#         547
  C:0647H         LINE#         548
  C:0652H         LINE#         549
  C:065DH         LINE#         550
  C:0668H         LINE#         551
  C:0671H         LINE#         552
  C:067AH         LINE#         553
  C:0683H         LINE#         554
  C:068CH         LINE#         555
  C:0697H         LINE#         556
  C:06A2H         LINE#         557
  C:06ABH         LINE#         558
  C:06B2H         LINE#         560
  C:06BDH         LINE#         561
  C:06C8H         LINE#         562
  C:06CFH         LINE#         564
  C:06DAH         LINE#         565
  C:06E1H         LINE#         567
  C:06ECH         LINE#         568
  C:06F7H         LINE#         569
  C:0702H         LINE#         570
  C:0709H         LINE#         572
  C:0712H         LINE#         573
  C:071BH         LINE#         577
  C:0724H         LINE#         578
  C:072FH         LINE#         579
  C:073AH         LINE#         580
  C:0745H         LINE#         581
  C:0750H         LINE#         582
  C:075BH         LINE#         583
  C:0766H         LINE#         584
  C:0771H         LINE#         585
BL51 BANKED LINKER/LOCATER V6.22                                                      12/05/2013  00:54:40  PAGE 16


  C:077CH         LINE#         586
  C:0787H         LINE#         590
  C:0790H         LINE#         591
  C:079BH         LINE#         592
  C:07A4H         LINE#         593
  C:07AFH         LINE#         595
  C:07B6H         LINE#         597
  C:07B6H         LINE#         598
  C:07B6H         LINE#         600
  C:07B9H         LINE#         601
  C:07C8H         LINE#         602
  C:07C8H         LINE#         603
  C:07D0H         LINE#         604
  C:07DBH         LINE#         605
  C:07E6H         LINE#         610
  C:07EFH         LINE#         611
  C:07FAH         LINE#         612
  C:0803H         LINE#         613
  C:080CH         LINE#         614
  C:0815H         LINE#         615
  C:081EH         LINE#         616
  C:0827H         LINE#         617
  C:082EH         LINE#         619
  C:0839H         LINE#         620
  C:0844H         LINE#         621
  C:084FH         LINE#         622
  C:085AH         LINE#         623
  C:0865H         LINE#         624
  C:0870H         LINE#         625
  C:087BH         LINE#         626
  C:0884H         LINE#         627
  C:088DH         LINE#         628
  C:0898H         LINE#         629
  C:08A1H         LINE#         630
  C:08ACH         LINE#         631
  C:08B7H         LINE#         633
  C:08C2H         LINE#         634
  C:08CBH         LINE#         635
  C:08D4H         LINE#         636
  C:08DDH         LINE#         637
  C:08E6H         LINE#         638
  C:08EFH         LINE#         639
  C:08F8H         LINE#         640
  C:0901H         LINE#         641
  C:090CH         LINE#         642
  C:0915H         LINE#         643
  C:0920H         LINE#         644
  C:092BH         LINE#         645
  C:0936H         LINE#         646
  C:0938H         LINE#         647
  C:0938H         LINE#         649
  C:094AH         LINE#         650
  C:094AH         LINE#         651
  C:0950H         LINE#         652
  C:0956H         LINE#         653
  C:095DH         LINE#         654
  C:0964H         LINE#         655
BL51 BANKED LINKER/LOCATER V6.22                                                      12/05/2013  00:54:40  PAGE 17


  C:096BH         LINE#         656
  C:0972H         LINE#         657
  C:0979H         LINE#         658
  C:0980H         LINE#         659
  C:0987H         LINE#         660
  C:098EH         LINE#         661
  C:0995H         LINE#         662
  C:099CH         LINE#         663
  C:09A3H         LINE#         664
  C:09AAH         LINE#         665
  C:09B1H         LINE#         666
  C:09B8H         LINE#         667
  C:09BEH         LINE#         668
  C:09C5H         LINE#         669
  C:09CCH         LINE#         670
  C:09D3H         LINE#         671
  C:09DAH         LINE#         672
  C:09E1H         LINE#         673
  C:09E7H         LINE#         674
  C:09EDH         LINE#         675
  C:09F4H         LINE#         676
  C:09FBH         LINE#         677
  C:0A02H         LINE#         678
  C:0A09H         LINE#         679
  C:0A10H         LINE#         680
  C:0A17H         LINE#         681
  C:0A1EH         LINE#         682
  C:0A25H         LINE#         683
  C:0A2CH         LINE#         684
  C:0A33H         LINE#         685
  C:0A3AH         LINE#         686
  C:0A41H         LINE#         687
  C:0A48H         LINE#         688
  C:0A4FH         LINE#         689
  C:0A55H         LINE#         690
  C:0A5CH         LINE#         691
  C:0A63H         LINE#         692
  C:0A6AH         LINE#         693
  C:0A71H         LINE#         694
  C:0A78H         LINE#         695
  C:0A7EH         LINE#         696
  C:0A85H         LINE#         697
  C:0A8CH         LINE#         698
  C:0A93H         LINE#         699
  C:0A9AH         LINE#         700
  C:0AA1H         LINE#         701
  C:0AA8H         LINE#         702
  C:0AAFH         LINE#         703
  C:0AB6H         LINE#         704
  C:0ABDH         LINE#         705
  C:0AC4H         LINE#         706
  C:0ACBH         LINE#         707
  C:0AD2H         LINE#         708
  C:0AD9H         LINE#         709
  C:0AE0H         LINE#         710
  C:0AE6H         LINE#         711
  C:0AECH         LINE#         712
BL51 BANKED LINKER/LOCATER V6.22                                                      12/05/2013  00:54:40  PAGE 18


  C:0AF2H         LINE#         713
  C:0AF8H         LINE#         714
  C:0AFFH         LINE#         715
  C:0B05H         LINE#         716
  C:0B0CH         LINE#         717
  C:0B13H         LINE#         718
  C:0B1AH         LINE#         719
  C:0B21H         LINE#         720
  C:0B28H         LINE#         721
  C:0B2FH         LINE#         722
  C:0B36H         LINE#         723
  C:0B3DH         LINE#         724
  C:0B44H         LINE#         725
  C:0B4BH         LINE#         726
  C:0B52H         LINE#         727
  C:0B59H         LINE#         728
  C:0B60H         LINE#         729
  C:0B67H         LINE#         730
  C:0B6EH         LINE#         731
  C:0B74H         LINE#         732
  C:0B7AH         LINE#         733
  C:0B81H         LINE#         734
  C:0B88H         LINE#         735
  C:0B8FH         LINE#         736
  C:0B95H         LINE#         737
  C:0B9BH         LINE#         738
  C:0BA1H         LINE#         739
  C:0BA8H         LINE#         740
  C:0BABH         LINE#         741
  C:0BB2H         LINE#         742
  C:0BB6H         LINE#         743
  C:0BB6H         LINE#         745
  C:0BB9H         LINE#         746
  C:0BC8H         LINE#         747
  C:0BC8H         LINE#         748
  C:0BCEH         LINE#         749
  C:0BD7H         LINE#         750
  C:0BE0H         LINE#         751
  C:0BE9H         LINE#         752
  C:0BF0H         LINE#         755
  C:0BFBH         LINE#         756
  C:0C04H         LINE#         757
  C:0C0FH         LINE#         758
  C:0C1AH         LINE#         759
  C:0C25H         LINE#         761
  C:0C30H         LINE#         762
  C:0C3BH         LINE#         763
  C:0C42H         LINE#         765
  C:0C4DH         LINE#         766
  C:0C58H         LINE#         767
  C:0C5FH         LINE#         770
  C:0C6AH         LINE#         771
  C:0C75H         LINE#         772
  C:0C80H         LINE#         773
  C:0C8BH         LINE#         774
  C:0C96H         LINE#         775
  C:0CA1H         LINE#         776
BL51 BANKED LINKER/LOCATER V6.22                                                      12/05/2013  00:54:40  PAGE 19


  C:0CACH         LINE#         777
  C:0CB7H         LINE#         778
  C:0CC2H         LINE#         779
  C:0CCDH         LINE#         780
  C:0CD8H         LINE#         781
  C:0CE3H         LINE#         782
  C:0CEAH         LINE#         785
  C:0CF5H         LINE#         786
  C:0D00H         LINE#         787
  C:0D0BH         LINE#         788
  C:0D14H         LINE#         789
  C:0D1FH         LINE#         790
  C:0D2AH         LINE#         791
  C:0D35H         LINE#         792
  C:0D3EH         LINE#         793
  C:0D49H         LINE#         794
  C:0D52H         LINE#         795
  C:0D5DH         LINE#         796
  C:0D66H         LINE#         797
  C:0D71H         LINE#         798
  C:0D7CH         LINE#         799
  C:0D87H         LINE#         800
  C:0D90H         LINE#         801
  C:0D97H         LINE#         804
  C:0D9AH         LINE#         805
  C:0DA5H         LINE#         806
  C:0DB0H         LINE#         807
  C:0DBBH         LINE#         809
  C:0DBFH         LINE#         811
  C:0DBFH         LINE#         813
  C:0DC2H         LINE#         814
  C:0DD1H         LINE#         815
  C:0DD1H         LINE#         817
  C:0DDAH         LINE#         818
  C:0DE4H         LINE#         819
  C:0DEBH         LINE#         820
  C:0DF6H         LINE#         821
  C:0E01H         LINE#         822
  C:0E0CH         LINE#         823
  C:0E15H         LINE#         824
  C:0E20H         LINE#         825
  C:0E29H         LINE#         826
  C:0E32H         LINE#         827
  C:0E3BH         LINE#         828
  C:0E44H         LINE#         829
  C:0E4DH         LINE#         831
  C:0E56H         LINE#         832
  C:0E5FH         LINE#         833
  C:0E68H         LINE#         834
  C:0E71H         LINE#         835
  C:0E78H         LINE#         836
  C:0E83H         LINE#         837
  C:0E8EH         LINE#         838
  C:0E95H         LINE#         839
  C:0EA0H         LINE#         840
  C:0EA7H         LINE#         841
  C:0EB2H         LINE#         842
BL51 BANKED LINKER/LOCATER V6.22                                                      12/05/2013  00:54:40  PAGE 20


  C:0EBDH         LINE#         843
  C:0EC4H         LINE#         844
  C:0ECDH         LINE#         845
  C:0ED6H         LINE#         847
  C:0EE1H         LINE#         848
  C:0EECH         LINE#         849
  C:0EF7H         LINE#         852
  C:0F02H         LINE#         853
  C:0F0DH         LINE#         854
  C:0F18H         LINE#         855
  C:0F23H         LINE#         856
  C:0F2EH         LINE#         857
  C:0F39H         LINE#         858
  C:0F44H         LINE#         860
  C:0F4DH         LINE#         861
  C:0F58H         LINE#         862
  C:0F61H         LINE#         863
  C:0F6CH         LINE#         864
  C:0F77H         LINE#         865
  C:0F82H         LINE#         866
  C:0F8BH         LINE#         868
  C:0F96H         LINE#         869
  C:0F9FH         LINE#         870
  C:0FAAH         LINE#         871
  C:0FB5H         LINE#         872
  C:0FBEH         LINE#         873
  C:0FC7H         LINE#         875
  C:0FD2H         LINE#         876
  C:0FD9H         LINE#         877
  C:0FE4H         LINE#         878
  C:0FEBH         LINE#         879
  C:0FF6H         LINE#         880
  C:0FFAH         LINE#         882
  C:0FFAH         LINE#         884
  C:0FFDH         LINE#         885
  C:100CH         LINE#         886
  C:100CH         LINE#         887
  C:1017H         LINE#         888
  C:1025H         LINE#         889
  C:1031H         LINE#         890
  C:103FH         LINE#         891
  C:104DH         LINE#         892
  C:105BH         LINE#         893
  C:1069H         LINE#         894
  C:1077H         LINE#         895
  C:1083H         LINE#         896
  C:1091H         LINE#         897
  C:109DH         LINE#         898
  C:10A9H         LINE#         899
  C:10B7H         LINE#         900
  C:10C5H         LINE#         901
  C:10D3H         LINE#         902
  C:10DFH         LINE#         903
  C:10EBH         LINE#         904
  C:10F7H         LINE#         905
  C:1103H         LINE#         906
  C:110FH         LINE#         907
BL51 BANKED LINKER/LOCATER V6.22                                                      12/05/2013  00:54:40  PAGE 21


  C:111DH         LINE#         908
  C:1129H         LINE#         909
  C:1135H         LINE#         910
  C:1143H         LINE#         911
  C:114FH         LINE#         912
  C:115DH         LINE#         913
  C:116BH         LINE#         914
  C:1179H         LINE#         915
  C:1187H         LINE#         916
  C:1195H         LINE#         917
  C:11A3H         LINE#         918
  C:11B1H         LINE#         919
  C:11BFH         LINE#         920
  C:11CDH         LINE#         921
  C:11DBH         LINE#         922
  C:11E9H         LINE#         923
  C:11F5H         LINE#         924
  C:1201H         LINE#         925
  C:1210H         LINE#         926
  C:1210H         LINE#         928
  C:121FH         LINE#         929
  C:121FH         LINE#         930
  C:121FH         LINE#         931
  C:121FH         LINE#         932
  C:121FH         LINE#         933
  C:121FH         LINE#         934
  C:121FH         LINE#         935
  C:121FH         LINE#         936
  C:121FH         LINE#         937
  C:121FH         LINE#         938
  C:121FH         LINE#         939
  C:121FH         LINE#         940
  C:121FH         LINE#         942
  C:121FH         LINE#         943
  C:121FH         LINE#         944
  C:121FH         LINE#         945
  C:121FH         LINE#         946
  C:121FH         LINE#         948
  C:121FH         LINE#         949
  C:121FH         LINE#         952
  C:121FH         LINE#         955
  C:121FH         LINE#         958
  C:121FH         LINE#         959
  C:121FH         LINE#         961
  C:121FH         LINE#         962
  C:121FH         LINE#         963
  C:121FH         LINE#         964
  C:121FH         LINE#         965
  C:121FH         LINE#         966
  C:121FH         LINE#         967
  C:121FH         LINE#         968
  C:121FH         LINE#         969
  C:121FH         LINE#         970
  C:121FH         LINE#         972
  C:121FH         LINE#         973
  C:121FH         LINE#         974
  C:121FH         LINE#         975
BL51 BANKED LINKER/LOCATER V6.22                                                      12/05/2013  00:54:40  PAGE 22


  C:121FH         LINE#         976
  C:121FH         LINE#         977
  C:121FH         LINE#         978
  C:121FH         LINE#         980
  C:121FH         LINE#         981
  C:121FH         LINE#         982
  C:121FH         LINE#         983
  C:121FH         LINE#         984
  C:121FH         LINE#         985
  C:121FH         LINE#         987
  C:121FH         LINE#         988
  C:121FH         LINE#         990
  C:121FH         LINE#         991
  C:121FH         LINE#         992
  C:121FH         LINE#         994
  C:1230H         LINE#         995
  C:1230H         LINE#         996
  C:123AH         LINE#         997
  C:1245H         LINE#         998
  C:1250H         LINE#         999
  C:125BH         LINE#         1000
  C:1264H         LINE#         1001
  C:126FH         LINE#         1002
  C:1278H         LINE#         1003
  C:1281H         LINE#         1004
  C:128AH         LINE#         1005
  C:1293H         LINE#         1006
  C:129CH         LINE#         1008
  C:12A5H         LINE#         1009
  C:12B0H         LINE#         1010
  C:12B9H         LINE#         1011
  C:12C2H         LINE#         1012
  C:12CBH         LINE#         1014
  C:12D6H         LINE#         1015
  C:12E1H         LINE#         1018
  C:12ECH         LINE#         1021
  C:12F7H         LINE#         1024
  C:1302H         LINE#         1025
  C:130DH         LINE#         1027
  C:1318H         LINE#         1028
  C:1323H         LINE#         1029
  C:132EH         LINE#         1030
  C:1339H         LINE#         1031
  C:1344H         LINE#         1032
  C:134FH         LINE#         1033
  C:135AH         LINE#         1034
  C:1365H         LINE#         1035
  C:1370H         LINE#         1036
  C:137BH         LINE#         1038
  C:1384H         LINE#         1039
  C:138FH         LINE#         1040
  C:1398H         LINE#         1041
  C:13A3H         LINE#         1042
  C:13AEH         LINE#         1043
  C:13B9H         LINE#         1044
  C:13C2H         LINE#         1046
  C:13CBH         LINE#         1047
BL51 BANKED LINKER/LOCATER V6.22                                                      12/05/2013  00:54:40  PAGE 23


  C:13D4H         LINE#         1048
  C:13DDH         LINE#         1049
  C:13E6H         LINE#         1050
  C:13EFH         LINE#         1051
  C:13F8H         LINE#         1053
  C:1403H         LINE#         1054
  C:140EH         LINE#         1056
  C:1416H         LINE#         1057
  C:1416H         LINE#         1058
  C:1416H         LINE#         1059
  C:1419H         LINE#         1060
  C:1428H         LINE#         1061
  C:1428H         LINE#         1062
  C:1432H         LINE#         1063
  C:143DH         LINE#         1066
  C:1448H         LINE#         1067
  C:1453H         LINE#         1068
  C:145EH         LINE#         1069
  C:1467H         LINE#         1070
  C:1472H         LINE#         1071
  C:147BH         LINE#         1072
  C:1484H         LINE#         1073
  C:148FH         LINE#         1074
  C:1498H         LINE#         1075
  C:14A1H         LINE#         1077
  C:14AAH         LINE#         1078
  C:14B5H         LINE#         1079
  C:14BEH         LINE#         1080
  C:14C7H         LINE#         1081
  C:14CAH         LINE#         1082
  C:14D1H         LINE#         1083
  C:14DCH         LINE#         1084
  C:14E7H         LINE#         1085
  C:14EEH         LINE#         1086
  C:14F9H         LINE#         1087
  C:1500H         LINE#         1088
  C:150BH         LINE#         1089
  C:1516H         LINE#         1090
  C:1521H         LINE#         1091
  C:1528H         LINE#         1092
  C:1531H         LINE#         1093
  C:153AH         LINE#         1094
  C:1541H         LINE#         1096
  C:154AH         LINE#         1097
  C:1555H         LINE#         1098
  C:1560H         LINE#         1099
  C:1569H         LINE#         1100
  C:1574H         LINE#         1101
  C:157FH         LINE#         1102
  C:158AH         LINE#         1103
  C:1595H         LINE#         1104
  C:159EH         LINE#         1105
  C:15A9H         LINE#         1106
  C:15B0H         LINE#         1107
  C:15B9H         LINE#         1108
  C:15C4H         LINE#         1109
  C:15CDH         LINE#         1110
BL51 BANKED LINKER/LOCATER V6.22                                                      12/05/2013  00:54:40  PAGE 24


  C:15D8H         LINE#         1112
  C:15E3H         LINE#         1113
  C:15EEH         LINE#         1114
  C:15F7H         LINE#         1115
  C:1600H         LINE#         1116
  C:1609H         LINE#         1117
  C:1612H         LINE#         1118
  C:161BH         LINE#         1119
  C:1624H         LINE#         1120
  C:162DH         LINE#         1122
  C:1638H         LINE#         1123
  C:1643H         LINE#         1125
  C:1643H         LINE#         1126
  C:1643H         LINE#         1128
  C:1655H         LINE#         1129
  C:1655H         LINE#         1130
  C:165FH         LINE#         1131
  C:166AH         LINE#         1132
  C:1675H         LINE#         1133
  C:1680H         LINE#         1135
  C:168BH         LINE#         1136
  C:1694H         LINE#         1137
  C:169DH         LINE#         1138
  C:16A6H         LINE#         1139
  C:16AFH         LINE#         1140
  C:16B8H         LINE#         1142
  C:16C1H         LINE#         1143
  C:16CCH         LINE#         1144
  C:16D5H         LINE#         1145
  C:16DEH         LINE#         1146
  C:16E5H         LINE#         1147
  C:16F0H         LINE#         1148
  C:16FBH         LINE#         1149
  C:1702H         LINE#         1150
  C:170DH         LINE#         1151
  C:1714H         LINE#         1152
  C:171FH         LINE#         1153
  C:172AH         LINE#         1154
  C:1735H         LINE#         1155
  C:173CH         LINE#         1156
  C:1745H         LINE#         1157
  C:1750H         LINE#         1159
  C:1759H         LINE#         1160
  C:1764H         LINE#         1161
  C:176DH         LINE#         1162
  C:1778H         LINE#         1163
  C:1783H         LINE#         1164
  C:178EH         LINE#         1165
  C:1799H         LINE#         1166
  C:17A4H         LINE#         1167
  C:17AFH         LINE#         1168
  C:17BAH         LINE#         1170
  C:17C3H         LINE#         1171
  C:17CEH         LINE#         1172
  C:17D7H         LINE#         1173
  C:17E2H         LINE#         1174
  C:17EDH         LINE#         1175
BL51 BANKED LINKER/LOCATER V6.22                                                      12/05/2013  00:54:40  PAGE 25


  C:17F8H         LINE#         1176
  C:1801H         LINE#         1178
  C:180AH         LINE#         1179
  C:1813H         LINE#         1180
  C:181CH         LINE#         1181
  C:1825H         LINE#         1182
  C:182EH         LINE#         1183
  C:1837H         LINE#         1185
  C:1842H         LINE#         1186
  C:184DH         LINE#         1187
  C:184DH         LINE#         1188
  C:184DH         LINE#         1190
  C:185FH         LINE#         1191
  C:185FH         LINE#         1193
  C:1867H         LINE#         1194
  C:186EH         LINE#         1195
  C:1879H         LINE#         1196
  C:1884H         LINE#         1197
  C:188FH         LINE#         1198
  C:189AH         LINE#         1199
  C:18A5H         LINE#         1201
  C:18B0H         LINE#         1202
  C:18BBH         LINE#         1203
  C:18C6H         LINE#         1204
  C:18D1H         LINE#         1205
  C:18DCH         LINE#         1206
  C:18E7H         LINE#         1207
  C:18F2H         LINE#         1208
  C:18FDH         LINE#         1209
  C:1906H         LINE#         1210
  C:190FH         LINE#         1211
  C:191AH         LINE#         1212
  C:1923H         LINE#         1213
  C:192EH         LINE#         1214
  C:1937H         LINE#         1215
  C:193EH         LINE#         1216
  C:1941H         LINE#         1217
  C:194CH         LINE#         1218
  C:1953H         LINE#         1220
  C:195EH         LINE#         1221
  C:1969H         LINE#         1222
  C:1974H         LINE#         1223
  C:197FH         LINE#         1224
  C:1988H         LINE#         1225
  C:1993H         LINE#         1226
  C:199EH         LINE#         1228
  C:19A7H         LINE#         1229
  C:19B2H         LINE#         1230
  C:19BBH         LINE#         1231
  C:19C6H         LINE#         1233
  C:19D1H         LINE#         1234
  C:19DCH         LINE#         1235
  C:19E5H         LINE#         1236
  C:19EEH         LINE#         1238
  C:19F7H         LINE#         1239
  C:1A00H         LINE#         1240
  C:1A09H         LINE#         1241
BL51 BANKED LINKER/LOCATER V6.22                                                      12/05/2013  00:54:40  PAGE 26


  C:1A12H         LINE#         1242
  C:1A1BH         LINE#         1244
  C:1A26H         LINE#         1245
  C:1A31H         LINE#         1246
  C:1A3CH         LINE#         1247
  C:1A45H         LINE#         1248
  C:1A4EH         LINE#         1249
  C:1A57H         LINE#         1251
  C:1A62H         LINE#         1252
  C:1A6DH         LINE#         1253
  C:1A78H         LINE#         1254
  C:1A81H         LINE#         1255
  C:1A8AH         LINE#         1256
  C:1A93H         LINE#         1257
  C:1A9CH         LINE#         1258
  C:1AA5H         LINE#         1259
  C:1AB0H         LINE#         1260
  C:1AB7H         LINE#         1261
  C:1AC2H         LINE#         1262
  C:1AC9H         LINE#         1263
  C:1AD4H         LINE#         1264
  C:1ADBH         LINE#         1265
  C:1ADBH         LINE#         1267
  C:1AEDH         LINE#         1268
  C:1AEDH         LINE#         1269
  C:1AF4H         LINE#         1270
  C:1AFCH         LINE#         1271
  C:1B04H         LINE#         1272
  C:1B0CH         LINE#         1274
  C:1B17H         LINE#         1275
  C:1B1EH         LINE#         1276
  C:1B29H         LINE#         1277
  C:1B34H         LINE#         1279
  C:1B3FH         LINE#         1280
  C:1B4AH         LINE#         1281
  C:1B55H         LINE#         1282
  C:1B60H         LINE#         1283
  C:1B6BH         LINE#         1284
  C:1B76H         LINE#         1285
  C:1B81H         LINE#         1286
  C:1B8CH         LINE#         1287
  C:1B97H         LINE#         1288
  C:1BA2H         LINE#         1290
  C:1BADH         LINE#         1291
  C:1BB6H         LINE#         1292
  C:1BC1H         LINE#         1293
  C:1BCAH         LINE#         1294
  C:1BD3H         LINE#         1295
  C:1BDAH         LINE#         1297
  C:1BE5H         LINE#         1298
  C:1BF0H         LINE#         1299
  C:1BF7H         LINE#         1301
  C:1C02H         LINE#         1302
  C:1C09H         LINE#         1304
  C:1C14H         LINE#         1305
  C:1C1FH         LINE#         1306
  C:1C2AH         LINE#         1307
BL51 BANKED LINKER/LOCATER V6.22                                                      12/05/2013  00:54:40  PAGE 27


  C:1C31H         LINE#         1309
  C:1C3CH         LINE#         1310
  C:1C47H         LINE#         1311
  C:1C52H         LINE#         1312
  C:1C5DH         LINE#         1313
  C:1C66H         LINE#         1314
  C:1C6FH         LINE#         1315
  C:1C78H         LINE#         1316
  C:1C83H         LINE#         1317
  C:1C8CH         LINE#         1318
  C:1C97H         LINE#         1319
  C:1CA0H         LINE#         1320
  C:1CABH         LINE#         1321
  C:1CB6H         LINE#         1322
  C:1CC1H         LINE#         1323
  C:1CCAH         LINE#         1326
  C:1CD5H         LINE#         1327
  C:1CE0H         LINE#         1328
  C:1CEBH         LINE#         1329
  C:1CF6H         LINE#         1330
  C:1CFDH         LINE#         1332
  C:1D00H         LINE#         1333
  C:1D07H         LINE#         1334
  C:1D12H         LINE#         1335
  C:1D1DH         LINE#         1337
  C:1D26H         LINE#         1338
  C:1D2FH         LINE#         1339
  C:1D39H         LINE#         1340
  C:1D39H         LINE#         1342
  C:1D4BH         LINE#         1343
  C:1D4BH         LINE#         1344
  C:1D52H         LINE#         1345
  C:1D5AH         LINE#         1346
  C:1D61H         LINE#         1347
  C:1D69H         LINE#         1348
  C:1D71H         LINE#         1349
  C:1D79H         LINE#         1350
  C:1D81H         LINE#         1351
  C:1D8CH         LINE#         1352
  C:1D93H         LINE#         1353
  C:1D9EH         LINE#         1354
  C:1DA9H         LINE#         1356
  C:1DB4H         LINE#         1357
  C:1DBFH         LINE#         1358
  C:1DCAH         LINE#         1359
  C:1DD5H         LINE#         1360
  C:1DE0H         LINE#         1361
  C:1DEBH         LINE#         1362
  C:1DF6H         LINE#         1363
  C:1E01H         LINE#         1364
  C:1E0CH         LINE#         1365
  C:1E17H         LINE#         1369
  C:1E22H         LINE#         1370
  C:1E2DH         LINE#         1371
  C:1E38H         LINE#         1372
  C:1E43H         LINE#         1373
  C:1E4EH         LINE#         1374
BL51 BANKED LINKER/LOCATER V6.22                                                      12/05/2013  00:54:40  PAGE 28


  C:1E55H         LINE#         1375
  C:1E60H         LINE#         1376
  C:1E6BH         LINE#         1377
  C:1E76H         LINE#         1379
  C:1E81H         LINE#         1380
  C:1E8AH         LINE#         1382
  C:1E95H         LINE#         1383
  C:1E9EH         LINE#         1384
  C:1EA7H         LINE#         1385
  C:1EB0H         LINE#         1386
  C:1EBBH         LINE#         1387
  C:1EC2H         LINE#         1388
  C:1ECDH         LINE#         1389
  C:1ED6H         LINE#         1390
  C:1EE1H         LINE#         1391
  C:1EEAH         LINE#         1392
  C:1EF5H         LINE#         1393
  C:1EFEH         LINE#         1394
  C:1F07H         LINE#         1395
  C:1F12H         LINE#         1397
  C:1F1DH         LINE#         1398
  C:1F28H         LINE#         1399
  C:1F28H         LINE#         1401
  C:1F3AH         LINE#         1402
  C:1F3AH         LINE#         1403
  C:1F42H         LINE#         1404
  C:1F49H         LINE#         1405
  C:1F54H         LINE#         1406
  C:1F5FH         LINE#         1407
  C:1F6AH         LINE#         1408
  C:1F71H         LINE#         1409
  C:1F7CH         LINE#         1410
  C:1F87H         LINE#         1411
  C:1F8EH         LINE#         1412
  C:1F99H         LINE#         1413
  C:1FA0H         LINE#         1414
  C:1FABH         LINE#         1415
  C:1FB6H         LINE#         1416
  C:1FBDH         LINE#         1417
  C:1FC8H         LINE#         1418
  C:1FD3H         LINE#         1419
  C:1FDEH         LINE#         1420
  C:1FE9H         LINE#         1421
  C:1FF4H         LINE#         1422
  C:1FFDH         LINE#         1423
  C:2008H         LINE#         1424
  C:2013H         LINE#         1425
  C:201EH         LINE#         1426
  C:2029H         LINE#         1427
  C:2034H         LINE#         1428
  C:203FH         LINE#         1429
  C:204AH         LINE#         1430
  C:2055H         LINE#         1431
  C:2060H         LINE#         1432
  C:206BH         LINE#         1433
  C:2076H         LINE#         1434
  C:2081H         LINE#         1435
BL51 BANKED LINKER/LOCATER V6.22                                                      12/05/2013  00:54:40  PAGE 29


  C:208CH         LINE#         1436
  C:2097H         LINE#         1437
  C:20A2H         LINE#         1438
  C:20ADH         LINE#         1439
  C:20B0H         LINE#         1440
  C:20BBH         LINE#         1441
  C:20C6H         LINE#         1442
  C:20D1H         LINE#         1443
  C:20DCH         LINE#         1444
  C:20E5H         LINE#         1445
  C:20E5H         LINE#         1447
  C:20F7H         LINE#         1448
  C:20F7H         LINE#         1449
  C:2100H         LINE#         1450
  C:210BH         LINE#         1451
  C:2116H         LINE#         1452
  C:2121H         LINE#         1453
  C:212CH         LINE#         1454
  C:2137H         LINE#         1455
  C:213EH         LINE#         1456
  C:2149H         LINE#         1457
  C:2150H         LINE#         1458
  C:215BH         LINE#         1459
  C:2166H         LINE#         1460
  C:216DH         LINE#         1461
  C:2176H         LINE#         1462
  C:2181H         LINE#         1463
  C:218CH         LINE#         1464
  C:2197H         LINE#         1465
  C:21A2H         LINE#         1466
  C:21ADH         LINE#         1467
  C:21B8H         LINE#         1468
  C:21C3H         LINE#         1469
  C:21CEH         LINE#         1470
  C:21D9H         LINE#         1472
  C:21E4H         LINE#         1473
  C:21EFH         LINE#         1474
  C:21FAH         LINE#         1475
  C:2204H         LINE#         1476
  C:220FH         LINE#         1477
  C:221AH         LINE#         1478
  C:2225H         LINE#         1479
  C:2230H         LINE#         1480
  C:223BH         LINE#         1481
  C:2246H         LINE#         1482
  C:2251H         LINE#         1483
  C:225CH         LINE#         1484
  C:225FH         LINE#         1485
  C:226AH         LINE#         1486
  C:2275H         LINE#         1487
  C:2280H         LINE#         1488
  C:228BH         LINE#         1489
  C:228BH         LINE#         1491
  C:2299H         LINE#         1492
  C:2299H         LINE#         1493
  C:229BH         LINE#         1494
  C:22A1H         LINE#         1495
BL51 BANKED LINKER/LOCATER V6.22                                                      12/05/2013  00:54:40  PAGE 30


  C:22A3H         LINE#         1496
  C:22AAH         LINE#         1497
  C:22ACH         LINE#         1498
  C:22AEH         LINE#         1499
  C:22B0H         LINE#         1500
  C:22B2H         LINE#         1501
  C:22B9H         LINE#         1504
  C:22C4H         LINE#         1505
  C:22CFH         LINE#         1506
  C:22D8H         LINE#         1507
  C:22E3H         LINE#         1508
  C:22EEH         LINE#         1509
  C:22F9H         LINE#         1510
  C:2304H         LINE#         1511
  C:230FH         LINE#         1512
  C:231AH         LINE#         1513
  C:2325H         LINE#         1514
  C:2330H         LINE#         1515
  C:233BH         LINE#         1518
  C:2344H         LINE#         1519
  C:234DH         LINE#         1520
  C:2356H         LINE#         1521
  C:2361H         LINE#         1522
  C:236AH         LINE#         1523
  C:2373H         LINE#         1524
  C:237EH         LINE#         1525
  C:2389H         LINE#         1528
  C:2394H         LINE#         1529
  C:239FH         LINE#         1530
  C:23AAH         LINE#         1531
  C:23B5H         LINE#         1532
  C:23C0H         LINE#         1534
  C:23CBH         LINE#         1535
  C:23D6H         LINE#         1536
  C:23E1H         LINE#         1537
  C:23ECH         LINE#         1538
  C:23F7H         LINE#         1539
  C:2402H         LINE#         1541
  C:240DH         LINE#         1542
  C:2416H         LINE#         1543
  C:2421H         LINE#         1544
  C:242AH         LINE#         1545
  C:2431H         LINE#         1546
  C:243CH         LINE#         1547
  C:2447H         LINE#         1548
  C:2452H         LINE#         1549
  C:245DH         LINE#         1550
  C:2468H         LINE#         1553
  C:2473H         LINE#         1554
  C:247EH         LINE#         1555
  C:2485H         LINE#         1556
  C:2490H         LINE#         1557
  C:249BH         LINE#         1558
  C:24A4H         LINE#         1559
  C:24AFH         LINE#         1562
  C:24BAH         LINE#         1563
  C:24C5H         LINE#         1564
BL51 BANKED LINKER/LOCATER V6.22                                                      12/05/2013  00:54:40  PAGE 31


  C:24CCH         LINE#         1565
  C:24D7H         LINE#         1566
  C:24DEH         LINE#         1568
  C:24E9H         LINE#         1569
  C:24F0H         LINE#         1570
  C:24FBH         LINE#         1571
  C:2502H         LINE#         1572
  C:250DH         LINE#         1573
  C:2514H         LINE#         1576
  C:251FH         LINE#         1577
  C:252AH         LINE#         1578
  C:2531H         LINE#         1579
  C:253CH         LINE#         1580
  C:2547H         LINE#         1581
  C:254EH         LINE#         1582
  C:2559H         LINE#         1585
  C:2564H         LINE#         1586
  C:256FH         LINE#         1587
  C:2578H         LINE#         1589
  C:257FH         LINE#         1590
  C:2586H         LINE#         1592
  C:2591H         LINE#         1593
  C:2591H         LINE#         1594
  C:2593H         LINE#         1595
  C:2599H         LINE#         1596
  C:259BH         LINE#         1597
  C:25A2H         LINE#         1598
  C:25A4H         LINE#         1599
  C:25A6H         LINE#         1600
  C:25A8H         LINE#         1601
  C:25AAH         LINE#         1602
  C:25B1H         LINE#         1605
  C:25BCH         LINE#         1606
  C:25C7H         LINE#         1607
  C:25D0H         LINE#         1608
  C:25DBH         LINE#         1609
  C:25E6H         LINE#         1610
  C:25F1H         LINE#         1611
  C:25FCH         LINE#         1612
  C:2607H         LINE#         1613
  C:2612H         LINE#         1614
  C:261DH         LINE#         1615
  C:2628H         LINE#         1616
  C:2633H         LINE#         1619
  C:263CH         LINE#         1620
  C:2645H         LINE#         1621
  C:264EH         LINE#         1622
  C:2659H         LINE#         1623
  C:2662H         LINE#         1624
  C:266BH         LINE#         1625
  C:2676H         LINE#         1626
  C:2681H         LINE#         1629
  C:268CH         LINE#         1630
  C:2697H         LINE#         1631
  C:26A2H         LINE#         1632
  C:26ADH         LINE#         1633
  C:26B8H         LINE#         1635
BL51 BANKED LINKER/LOCATER V6.22                                                      12/05/2013  00:54:40  PAGE 32


  C:26C3H         LINE#         1636
  C:26CEH         LINE#         1637
  C:26D9H         LINE#         1638
  C:26E4H         LINE#         1639
  C:26EFH         LINE#         1640
  C:26FAH         LINE#         1642
  C:2705H         LINE#         1643
  C:270EH         LINE#         1644
  C:2719H         LINE#         1645
  C:2722H         LINE#         1646
  C:2729H         LINE#         1647
  C:2734H         LINE#         1648
  C:273FH         LINE#         1649
  C:274AH         LINE#         1650
  C:2755H         LINE#         1651
  C:2760H         LINE#         1654
  C:276BH         LINE#         1655
  C:2776H         LINE#         1656
  C:277DH         LINE#         1657
  C:2788H         LINE#         1658
  C:2793H         LINE#         1659
  C:279CH         LINE#         1660
  C:27A7H         LINE#         1663
  C:27B2H         LINE#         1664
  C:27BDH         LINE#         1665
  C:27C4H         LINE#         1666
  C:27CFH         LINE#         1667
  C:27D6H         LINE#         1669
  C:27E1H         LINE#         1670
  C:27E8H         LINE#         1671
  C:27F3H         LINE#         1672
  C:27FAH         LINE#         1673
  C:2805H         LINE#         1674
  C:280CH         LINE#         1677
  C:2817H         LINE#         1678
  C:2822H         LINE#         1679
  C:2829H         LINE#         1680
  C:2834H         LINE#         1681
  C:283FH         LINE#         1682
  C:2846H         LINE#         1683
  C:2851H         LINE#         1686
  C:285CH         LINE#         1687
  C:2867H         LINE#         1688
  C:2870H         LINE#         1690
  C:2877H         LINE#         1691
  C:2877H         LINE#         1693
  -------         ENDPROC       LCD_INIT
  -------         PROC          _LCD_ID
  D:0008H         SYMBOL        dat
  -------         DO            
  D:000AH         SYMBOL        temp
  D:000CH         SYMBOL        DH
  D:000EH         SYMBOL        DL
  D:000AH         SYMBOL        temp
  D:000CH         SYMBOL        DH
  D:000EH         SYMBOL        DL
  -------         ENDDO         
BL51 BANKED LINKER/LOCATER V6.22                                                      12/05/2013  00:54:40  PAGE 33


  -------         DO            
  D:000AH         SYMBOL        temp
  D:000CH         SYMBOL        DH
  D:000EH         SYMBOL        DL
  -------         ENDDO         
  C:3EBDH         LINE#         1699
  C:3EC1H         LINE#         1700
  C:3EC1H         LINE#         1701
  C:3EC9H         LINE#         1702
  C:3EC9H         LINE#         1704
  C:3ECDH         LINE#         1705
  C:3ED0H         LINE#         1706
  C:3ED5H         LINE#         1707
  C:3ED8H         LINE#         1708
  C:3EDBH         LINE#         1710
  C:3EDDH         LINE#         1711
  C:3EDFH         LINE#         1712
  C:3EE1H         LINE#         1713
  C:3EE7H         LINE#         1714
  C:3EEEH         LINE#         1716
  C:3EF0H         LINE#         1717
  C:3EF2H         LINE#         1718
  C:3EF9H         LINE#         1722
  C:3EFBH         LINE#         1723
  C:3EFDH         LINE#         1724
  C:3F03H         LINE#         1726
  C:3F03H         LINE#         1727
  C:3F03H         LINE#         1728
  C:3F03H         LINE#         1730
  C:3F05H         LINE#         1731
  C:3F05H         LINE#         1732
  C:3F05H         LINE#         1734
  C:3F0CH         LINE#         1735
  C:3F11H         LINE#         1736
  C:3F14H         LINE#         1737
  C:3F17H         LINE#         1739
  C:3F19H         LINE#         1740
  C:3F1BH         LINE#         1741
  C:3F1DH         LINE#         1742
  C:3F23H         LINE#         1744
  C:3F2AH         LINE#         1745
  C:3F31H         LINE#         1748
  C:3F33H         LINE#         1752
  C:3F35H         LINE#         1754
  C:3F3DH         LINE#         1755
  C:3F44H         LINE#         1756
  C:3F4CH         LINE#         1758
  C:3F50H         LINE#         1759
  C:3F50H         LINE#         1760
  -------         ENDPROC       _LCD_ID
  -------         PROC          _LCD_ID_61581
  D:0008H         SYMBOL        dat
  -------         DO            
  D:000AH         SYMBOL        temp
  D:0006H         SYMBOL        DH
  D:0004H         SYMBOL        DL
  -------         ENDDO         
BL51 BANKED LINKER/LOCATER V6.22                                                      12/05/2013  00:54:40  PAGE 34


  C:3C6BH         LINE#         1765
  C:3C6FH         LINE#         1766
  C:3C6FH         LINE#         1770
  C:3C76H         LINE#         1771
  C:3C7CH         LINE#         1773
  C:3C83H         LINE#         1774
  C:3C88H         LINE#         1775
  C:3C8BH         LINE#         1776
  C:3C8EH         LINE#         1778
  C:3C90H         LINE#         1779
  C:3C92H         LINE#         1780
  C:3C94H         LINE#         1781
  C:3C9AH         LINE#         1783
  C:3C9EH         LINE#         1784
  C:3CA2H         LINE#         1786
  C:3CA4H         LINE#         1787
  C:3CA7H         LINE#         1788
  C:3CACH         LINE#         1790
  C:3CAEH         LINE#         1791
  C:3CB0H         LINE#         1792
  C:3CB2H         LINE#         1793
  C:3CB7H         LINE#         1795
  C:3CBBH         LINE#         1796
  C:3CBFH         LINE#         1798
  C:3CC1H         LINE#         1799
  C:3CC4H         LINE#         1800
  C:3CC9H         LINE#         1802
  C:3CCBH         LINE#         1803
  C:3CCDH         LINE#         1804
  C:3CCFH         LINE#         1805
  C:3CD4H         LINE#         1807
  C:3CD8H         LINE#         1808
  C:3CDCH         LINE#         1810
  C:3CDEH         LINE#         1811
  C:3CE1H         LINE#         1812
  C:3CE6H         LINE#         1816
  C:3CE8H         LINE#         1817
  C:3CEAH         LINE#         1818
  C:3CECH         LINE#         1819
  C:3CF1H         LINE#         1821
  C:3CF5H         LINE#         1822
  C:3CF9H         LINE#         1824
  C:3CFBH         LINE#         1825
  C:3CFEH         LINE#         1826
  C:3D03H         LINE#         1828
  C:3D06H         LINE#         1829
  C:3D0DH         LINE#         1831
  C:3D0FH         LINE#         1832
  C:3D11H         LINE#         1833
  C:3D13H         LINE#         1834
  C:3D18H         LINE#         1836
  C:3D1AH         LINE#         1837
  C:3D1EH         LINE#         1839
  C:3D20H         LINE#         1840
  C:3D23H         LINE#         1841
  C:3D28H         LINE#         1845
  C:3D2AH         LINE#         1849
BL51 BANKED LINKER/LOCATER V6.22                                                      12/05/2013  00:54:40  PAGE 35


  C:3D2DH         LINE#         1851
  C:3D31H         LINE#         1852
  -------         ENDPROC       _LCD_ID_61581
  -------         PROC          LCD_READ_ID61581
  -------         DO            
  D:0005H         SYMBOL        m
  D:0004H         SYMBOL        n
  -------         ENDDO         
  C:42CFH         LINE#         1857
  C:42CFH         LINE#         1858
  C:42CFH         LINE#         1861
  C:42CFH         LINE#         1862
  C:42CFH         LINE#         1863
  C:42D2H         LINE#         1864
  C:42D9H         LINE#         1866
  C:42E4H         LINE#         1869
  C:42E6H         LINE#         1870
  C:42E6H         LINE#         1871
  C:42E6H         LINE#         1873
  C:42E6H         LINE#         1874
  C:42E6H         LINE#         1875
  C:42E6H         LINE#         1877
  C:42E9H         LINE#         1878
  -------         ENDPROC       LCD_READ_ID61581
  -------         PROC          _LCD_ID_9341
  D:0006H         SYMBOL        dat
  -------         DO            
  D:0008H         SYMBOL        temp
  D:000AH         SYMBOL        DH
  D:000CH         SYMBOL        DL
  -------         ENDDO         
  C:3FD4H         LINE#         1885
  C:3FD4H         LINE#         1886
  C:3FD4H         LINE#         1887
  C:3FDCH         LINE#         1888
  C:3FDCH         LINE#         1889
  C:3FE0H         LINE#         1890
  C:3FE0H         LINE#         1891
  C:3FE0H         LINE#         1893
  C:3FE3H         LINE#         1894
  C:3FE8H         LINE#         1895
  C:3FEBH         LINE#         1896
  C:3FEEH         LINE#         1898
  C:3FF0H         LINE#         1899
  C:3FF2H         LINE#         1900
  C:3FF4H         LINE#         1901
  C:3FFAH         LINE#         1903
  C:3FFAH         LINE#         1904
  C:3FFAH         LINE#         1906
  C:3FFAH         LINE#         1907
  C:3FFAH         LINE#         1908
  C:3FFAH         LINE#         1910
  C:3FFAH         LINE#         1911
  C:3FFAH         LINE#         1912
  C:3FFAH         LINE#         1913
  C:3FFDH         LINE#         1915
  C:3FFDH         LINE#         1916
BL51 BANKED LINKER/LOCATER V6.22                                                      12/05/2013  00:54:40  PAGE 36


  C:3FFDH         LINE#         1918
  C:3FFDH         LINE#         1919
  C:3FFDH         LINE#         1920
  C:3FFDH         LINE#         1922
  C:3FFDH         LINE#         1923
  C:3FFDH         LINE#         1924
  C:3FFDH         LINE#         1925
  C:4000H         LINE#         1927
  C:4007H         LINE#         1928
  C:400EH         LINE#         1930
  C:4010H         LINE#         1931
  C:4015H         LINE#         1932
  C:401AH         LINE#         1934
  C:4022H         LINE#         1935
  C:4029H         LINE#         1940
  C:4029H         LINE#         1941
  C:4029H         LINE#         1942
  C:4029H         LINE#         1943
  C:402CH         LINE#         1945
  C:4033H         LINE#         1946
  C:403AH         LINE#         1948
  C:403CH         LINE#         1949
  C:4041H         LINE#         1950
  C:4046H         LINE#         1954
  C:4048H         LINE#         1957
  C:4050H         LINE#         1959
  C:4054H         LINE#         1960
  C:4054H         LINE#         1961
  -------         ENDPROC       _LCD_ID_9341
  -------         PROC          LCD_READ_8347ID
  -------         DO            
  D:0005H         SYMBOL        m
  D:0004H         SYMBOL        n
  -------         ENDDO         
  C:420AH         LINE#         1966
  C:420AH         LINE#         1967
  C:420AH         LINE#         1970
  C:420AH         LINE#         1971
  C:420DH         LINE#         1972
  C:4214H         LINE#         1973
  C:421EH         LINE#         1974
  C:4225H         LINE#         1975
  C:422CH         LINE#         1976
  C:422CH         LINE#         1978
  C:422CH         LINE#         1979
  C:422CH         LINE#         1980
  C:422CH         LINE#         1982
  C:422CH         LINE#         1983
  C:422CH         LINE#         1984
  C:422CH         LINE#         1986
  C:422FH         LINE#         1987
  -------         ENDPROC       LCD_READ_8347ID
  -------         PROC          LCD_READ_ID
  -------         DO            
  D:0005H         SYMBOL        m
  D:0004H         SYMBOL        n
  -------         ENDDO         
BL51 BANKED LINKER/LOCATER V6.22                                                      12/05/2013  00:54:40  PAGE 37


  C:425DH         LINE#         1993
  C:425DH         LINE#         1994
  C:425DH         LINE#         1997
  C:425DH         LINE#         1998
  C:4260H         LINE#         1999
  C:4267H         LINE#         2000
  C:4271H         LINE#         2001
  C:4278H         LINE#         2002
  C:427EH         LINE#         2003
  C:427EH         LINE#         2005
  C:427EH         LINE#         2006
  C:427EH         LINE#         2007
  C:427EH         LINE#         2009
  C:427EH         LINE#         2010
  C:427EH         LINE#         2011
  C:427EH         LINE#         2013
  C:4281H         LINE#         2014
  -------         ENDPROC       LCD_READ_ID
  -------         PROC          LCD_READ_ID9341
  -------         DO            
  D:0005H         SYMBOL        m
  D:0004H         SYMBOL        n
  -------         ENDDO         
  C:4286H         LINE#         2020
  C:4286H         LINE#         2021
  C:4286H         LINE#         2024
  C:4286H         LINE#         2025
  C:4286H         LINE#         2026
  C:4289H         LINE#         2027
  C:4290H         LINE#         2028
  C:4297H         LINE#         2029
  C:42A2H         LINE#         2032
  C:42A4H         LINE#         2033
  C:42A4H         LINE#         2034
  C:42A4H         LINE#         2036
  C:42A4H         LINE#         2037
  C:42A4H         LINE#         2038
  C:42A4H         LINE#         2040
  C:42A7H         LINE#         2041
  -------         ENDPROC       LCD_READ_ID9341
  C:434CH         SYMBOL        L?0383
  -------         PROC          L?0382
  -------         ENDPROC       L?0382
  C:434CH         SYMBOL        L?0383
  -------         PROC          HD_RESET
  C:4351H         LINE#         2048
  C:4351H         LINE#         2049
  C:4351H         LINE#         2050
  C:4353H         LINE#         2051
  C:435AH         LINE#         2052
  C:435CH         LINE#         2053
  -------         ENDPROC       HD_RESET
  -------         PROC          _LCD_WRITE_CMD
  D:0007H         SYMBOL        cmd1
  D:0005H         SYMBOL        cmd2
  C:41DDH         LINE#         2059
  C:41DDH         LINE#         2060
BL51 BANKED LINKER/LOCATER V6.22                                                      12/05/2013  00:54:40  PAGE 38


  C:41DDH         LINE#         2061
  C:41E5H         LINE#         2062
  C:41E5H         LINE#         2063
  C:41E7H         LINE#         2064
  C:41E9H         LINE#         2065
  C:41EBH         LINE#         2066
  C:41EDH         LINE#         2067
  C:41EFH         LINE#         2068
  C:41F1H         LINE#         2070
  C:41F3H         LINE#         2071
  C:41F5H         LINE#         2072
  C:41F5H         LINE#         2074
  C:41F5H         LINE#         2075
  C:41F5H         LINE#         2076
  C:41F7H         LINE#         2077
  C:41F7H         LINE#         2078
  C:41F9H         LINE#         2079
  C:41FBH         LINE#         2080
  C:41FDH         LINE#         2081
  C:41FFH         LINE#         2082
  C:4201H         LINE#         2084
  C:4203H         LINE#         2085
  C:4205H         LINE#         2087
  C:4207H         LINE#         2088
  C:4209H         LINE#         2089
  C:4209H         LINE#         2090
  -------         ENDPROC       _LCD_WRITE_CMD
  C:40B9H         SYMBOL        L?0379
  -------         PROC          L?0378
  -------         ENDPROC       L?0378
  C:40B9H         SYMBOL        L?0379
  -------         PROC          _LCD_WRITE_DATA
  D:0007H         SYMBOL        dataa
  D:0005H         SYMBOL        datab
  C:40BEH         LINE#         2095
  C:40BEH         LINE#         2096
  C:40BEH         LINE#         2097
  C:40C6H         LINE#         2098
  C:40C6H         LINE#         2099
  C:40C8H         LINE#         2100
  C:40CAH         LINE#         2101
  C:40CCH         LINE#         2102
  C:40CEH         LINE#         2103
  C:40D0H         LINE#         2104
  C:40D2H         LINE#         2106
  C:40D4H         LINE#         2107
  C:40D6H         LINE#         2108
  C:40D6H         LINE#         2110
  C:40D6H         LINE#         2111
  C:40D6H         LINE#         2112
  C:40D8H         LINE#         2113
  C:40D8H         LINE#         2114
  C:40DAH         LINE#         2115
  C:40DCH         LINE#         2116
  C:40DEH         LINE#         2117
  C:40E0H         LINE#         2118
  C:40E2H         LINE#         2120
BL51 BANKED LINKER/LOCATER V6.22                                                      12/05/2013  00:54:40  PAGE 39


  C:40E4H         LINE#         2121
  C:40E6H         LINE#         2123
  C:40E8H         LINE#         2124
  C:40EAH         LINE#         2125
  C:40EAH         LINE#         2126
  -------         ENDPROC       _LCD_WRITE_DATA
  C:416CH         SYMBOL        L?0381
  -------         PROC          L?0380
  -------         ENDPROC       L?0380
  C:416CH         SYMBOL        L?0381
  -------         PROC          _LLCD_WRITE_CMD
  D:0004H         SYMBOL        cmd
  C:4170H         LINE#         2131
  C:4174H         LINE#         2132
  C:4174H         LINE#         2133
  C:417CH         LINE#         2134
  C:417CH         LINE#         2135
  C:417EH         LINE#         2136
  C:4180H         LINE#         2137
  C:4182H         LINE#         2138
  C:4184H         LINE#         2139
  C:4188H         LINE#         2140
  C:418AH         LINE#         2142
  C:418CH         LINE#         2143
  C:418EH         LINE#         2144
  C:418EH         LINE#         2146
  C:418EH         LINE#         2147
  C:418EH         LINE#         2148
  C:4190H         LINE#         2149
  C:4190H         LINE#         2150
  C:4192H         LINE#         2151
  C:4194H         LINE#         2152
  C:4196H         LINE#         2153
  C:4198H         LINE#         2154
  C:419CH         LINE#         2156
  C:419EH         LINE#         2157
  C:41A0H         LINE#         2159
  C:41A2H         LINE#         2160
  C:41A4H         LINE#         2161
  C:41A4H         LINE#         2162
  -------         ENDPROC       _LLCD_WRITE_CMD
  -------         PROC          L?0377
  -------         ENDPROC       L?0377
  -------         PROC          _LLCD_WRITE_DATA
  D:0004H         SYMBOL        dataa
  C:41A8H         LINE#         2167
  C:41ACH         LINE#         2168
  C:41ACH         LINE#         2169
  C:41B4H         LINE#         2170
  C:41B4H         LINE#         2171
  C:41B6H         LINE#         2172
  C:41B8H         LINE#         2173
  C:41BAH         LINE#         2174
  C:41BCH         LINE#         2175
  C:41C0H         LINE#         2176
  C:41C2H         LINE#         2178
  C:41C4H         LINE#         2179
BL51 BANKED LINKER/LOCATER V6.22                                                      12/05/2013  00:54:40  PAGE 40


  C:41C6H         LINE#         2180
  C:41C6H         LINE#         2182
  C:41C6H         LINE#         2183
  C:41C6H         LINE#         2184
  C:41C8H         LINE#         2185
  C:41C8H         LINE#         2186
  C:41CAH         LINE#         2187
  C:41CCH         LINE#         2188
  C:41CEH         LINE#         2189
  C:41D0H         LINE#         2190
  C:41D4H         LINE#         2195
  C:41D6H         LINE#         2196
  C:41D8H         LINE#         2198
  C:41DAH         LINE#         2199
  C:41DCH         LINE#         2200
  C:41DCH         LINE#         2201
  -------         ENDPROC       _LLCD_WRITE_DATA
  C:4363H         SYMBOL        L?0368
  C:4365H         SYMBOL        L?0369
  -------         PROC          L?0367
  -------         ENDPROC       L?0367
  C:4363H         SYMBOL        L?0368
  C:4365H         SYMBOL        L?0369
  -------         PROC          _SENG_CMD_DAT
  D:0006H         SYMBOL        cmd
  D:0002H         SYMBOL        dataa
  C:436BH         LINE#         2207
  C:436FH         LINE#         2208
  C:436FH         LINE#         2209
  C:4372H         LINE#         2210
  -------         ENDPROC       _SENG_CMD_DAT
  C:4059H         SYMBOL        L?0371
  -------         PROC          L?0370
  -------         ENDPROC       L?0370
  C:4059H         SYMBOL        L?0371
  -------         PROC          _GUI_SPRINTF_STRING
  D:0008H         SYMBOL        x
  D:0009H         SYMBOL        y
  D:000BH         SYMBOL        s
  D:000DH         SYMBOL        color
  D:000FH         SYMBOL        b_color
  C:4069H         LINE#         2216
  C:4073H         LINE#         2217
  C:4073H         LINE#         2218
  C:407EH         LINE#         2219
  C:407EH         LINE#         2220
  C:4093H         LINE#         2221
  C:4099H         LINE#         2222
  C:40A3H         LINE#         2225
  -------         ENDPROC       _GUI_SPRINTF_STRING
  -------         PROC          _GUI_SPRINTF_CHAR
  D:0011H         SYMBOL        x
  D:0012H         SYMBOL        y
  D:0014H         SYMBOL        c
  D:0015H         SYMBOL        color
  D:0017H         SYMBOL        b_color
  -------         DO            
BL51 BANKED LINKER/LOCATER V6.22                                                      12/05/2013  00:54:40  PAGE 41


  D:0019H         SYMBOL        s_x
  D:001AH         SYMBOL        s_y
  D:001BH         SYMBOL        temp
  D:0006H         SYMBOL        j
  -------         ENDDO         
  C:3DF9H         LINE#         2230
  C:3E01H         LINE#         2231
  C:3E01H         LINE#         2234
  C:3E07H         LINE#         2235
  C:3E0AH         LINE#         2236
  C:3E0AH         LINE#         2237
  C:3E22H         LINE#         2238
  C:3E22H         LINE#         2239
  C:3E26H         LINE#         2240
  C:3E3AH         LINE#         2241
  C:3E48H         LINE#         2243
  C:3E4BH         LINE#         2244
  C:3E4BH         LINE#         2245
  C:3E5EH         LINE#         2246
  C:3E5EH         LINE#         2247
  C:3E7CH         LINE#         2248
  C:3E7CH         LINE#         2249
  C:3E8EH         LINE#         2250
  C:3E90H         LINE#         2252
  C:3E90H         LINE#         2253
  C:3EA7H         LINE#         2254
  C:3EA7H         LINE#         2255
  C:3EA7H         LINE#         2256
  C:3EB0H         LINE#         2257
  C:3EB0H         LINE#         2258
  C:3EBCH         LINE#         2259
  -------         ENDPROC       _GUI_SPRINTF_CHAR
  -------         PROC          _GUI_POINT
  D:0007H         SYMBOL        x
  D:0004H         SYMBOL        y
  D:001CH         SYMBOL        color
  C:4388H         LINE#         2264
  C:438CH         LINE#         2265
  C:438CH         LINE#         2266
  C:438FH         LINE#         2267
  -------         ENDPROC       _GUI_POINT
  -------         PROC          _LCD_SETXY
  D:0003H         SYMBOL        x
  D:0004H         SYMBOL        y
  C:43C6H         LINE#         2273
  C:43C8H         LINE#         2274
  C:43C8H         LINE#         2275
  -------         ENDPROC       _LCD_SETXY
  -------         PROC          _LCD_SETWINDOW
  D:0001H         SYMBOL        x0
  D:001FH         SYMBOL        y0
  D:0021H         SYMBOL        x1
  D:0022H         SYMBOL        y1
  C:3A1FH         LINE#         2281
  C:3A27H         LINE#         2282
  C:3A27H         LINE#         2283
  C:3A32H         LINE#         2284
BL51 BANKED LINKER/LOCATER V6.22                                                      12/05/2013  00:54:40  PAGE 42


  C:3A3EH         LINE#         2285
  C:3A49H         LINE#         2286
  C:3A54H         LINE#         2287
  C:3A5EH         LINE#         2288
  C:3A5EH         LINE#         2289
  C:3A69H         LINE#         2290
  C:3A6FH         LINE#         2291
  C:3A6FH         LINE#         2292
  C:3A7EH         LINE#         2293
  C:3A7EH         LINE#         2294
  C:3A7EH         LINE#         2295
  C:3A7EH         LINE#         2296
  C:3A7EH         LINE#         2298
  C:3A7EH         LINE#         2299
  C:3A7EH         LINE#         2300
  C:3A7EH         LINE#         2302
  C:3A7EH         LINE#         2303
  C:3A8CH         LINE#         2304
  C:3A8CH         LINE#         2305
  C:3A92H         LINE#         2306
  C:3A97H         LINE#         2307
  C:3A9CH         LINE#         2309
  C:3AA1H         LINE#         2310
  C:3AA7H         LINE#         2311
  C:3AACH         LINE#         2313
  C:3AAEH         LINE#         2314
  C:3AB1H         LINE#         2315
  C:3ABDH         LINE#         2316
  C:3ABDH         LINE#         2317
  C:3AC8H         LINE#         2318
  C:3AD2H         LINE#         2319
  C:3ADEH         LINE#         2320
  C:3AECH         LINE#         2322
  C:3AF8H         LINE#         2323
  C:3B04H         LINE#         2324
  C:3B08H         LINE#         2325
  C:3B0AH         LINE#         2326
  C:3B12H         LINE#         2327
  C:3B12H         LINE#         2328
  C:3B1AH         LINE#         2329
  C:3B25H         LINE#         2330
  C:3B2EH         LINE#         2331
  C:3B3AH         LINE#         2332
  C:3B46H         LINE#         2333
  C:3B51H         LINE#         2334
  C:3B5DH         LINE#         2335
  C:3B63H         LINE#         2336
  C:3B63H         LINE#         2337
  C:3B65H         LINE#         2339
  C:3B65H         LINE#         2340
  C:3B70H         LINE#         2341
  C:3B7BH         LINE#         2342
  C:3B82H         LINE#         2343
  C:3B82H         LINE#         2345
  -------         ENDPROC       _LCD_SETWINDOW
  -------         PROC          _LCD_TEST_SINGLECOLOR
  D:0008H         SYMBOL        colorH
BL51 BANKED LINKER/LOCATER V6.22                                                      12/05/2013  00:54:40  PAGE 43


  D:0001H         SYMBOL        colorL
  -------         DO            
  D:0009H         SYMBOL        i
  D:0082H         SYMBOL        j
  -------         ENDDO         
  C:35ECH         LINE#         2350
  C:35F0H         LINE#         2351
  C:35F0H         LINE#         2353
  C:35FCH         LINE#         2354
  C:35FCH         LINE#         2355
  C:35FEH         LINE#         2356
  C:35FEH         LINE#         2357
  C:3601H         LINE#         2358
  C:360CH         LINE#         2360
  C:3612H         LINE#         2361
  C:3617H         LINE#         2362
  C:361CH         LINE#         2363
  C:3621H         LINE#         2366
  C:3628H         LINE#         2367
  C:362AH         LINE#         2368
  C:362AH         LINE#         2369
  C:3639H         LINE#         2370
  C:3639H         LINE#         2371
  C:3639H         LINE#         2372
  C:3639H         LINE#         2373
  C:3639H         LINE#         2374
  C:3639H         LINE#         2378
  C:3639H         LINE#         2379
  C:3639H         LINE#         2380
  C:3639H         LINE#         2381
  C:3647H         LINE#         2382
  C:3647H         LINE#         2383
  C:3650H         LINE#         2384
  C:3659H         LINE#         2385
  C:3663H         LINE#         2386
  C:366EH         LINE#         2390
  C:3674H         LINE#         2391
  C:3679H         LINE#         2392
  C:367BH         LINE#         2393
  C:368AH         LINE#         2394
  C:368AH         LINE#         2395
  C:3693H         LINE#         2396
  C:369EH         LINE#         2397
  C:36A8H         LINE#         2398
  C:36B3H         LINE#         2400
  C:36BCH         LINE#         2401
  C:36C6H         LINE#         2402
  C:36CAH         LINE#         2403
  C:36D9H         LINE#         2404
  C:36D9H         LINE#         2405
  C:36E1H         LINE#         2406
  C:36EAH         LINE#         2407
  C:36F5H         LINE#         2408
  C:3700H         LINE#         2409
  C:3709H         LINE#         2410
  C:3714H         LINE#         2411
  C:371DH         LINE#         2412
BL51 BANKED LINKER/LOCATER V6.22                                                      12/05/2013  00:54:40  PAGE 44


  C:3728H         LINE#         2413
  C:372CH         LINE#         2414
  C:373BH         LINE#         2415
  C:373BH         LINE#         2416
  C:3743H         LINE#         2417
  C:374CH         LINE#         2418
  C:3757H         LINE#         2419
  C:3762H         LINE#         2420
  C:376BH         LINE#         2421
  C:3776H         LINE#         2422
  C:377FH         LINE#         2423
  C:378AH         LINE#         2424
  C:378EH         LINE#         2425
  C:379CH         LINE#         2426
  C:379CH         LINE#         2427
  C:37A7H         LINE#         2428
  C:37B1H         LINE#         2429
  C:37BCH         LINE#         2430
  C:37C7H         LINE#         2432
  C:37D1H         LINE#         2433
  C:37DBH         LINE#         2434
  C:37E0H         LINE#         2436
  C:37E2H         LINE#         2439
  C:37E2H         LINE#         2440
  C:37E5H         LINE#         2441
  C:37E5H         LINE#         2442
  C:37E8H         LINE#         2443
  C:37F3H         LINE#         2447
  C:37F9H         LINE#         2448
  C:37FEH         LINE#         2449
  C:3803H         LINE#         2450
  C:3803H         LINE#         2452
  C:380DH         LINE#         2453
  C:380DH         LINE#         2454
  C:3812H         LINE#         2455
  C:3812H         LINE#         2456
  C:3817H         LINE#         2457
  C:3817H         LINE#         2458
  C:381EH         LINE#         2459
  C:3829H         LINE#         2460
  C:383DH         LINE#         2461
  C:383DH         LINE#         2462
  C:383DH         LINE#         2463
  C:3842H         LINE#         2464
  C:3842H         LINE#         2465
  C:3847H         LINE#         2466
  C:3847H         LINE#         2467
  C:384EH         LINE#         2468
  C:3857H         LINE#         2470
  -------         ENDPROC       _LCD_TEST_SINGLECOLOR
  -------         PROC          KEYPRESS
  C:4396H         LINE#         2486
  C:4396H         LINE#         2487
  C:4396H         LINE#         2488
  C:4399H         LINE#         2489
  C:43A2H         LINE#         2490
  -------         ENDPROC       KEYPRESS
BL51 BANKED LINKER/LOCATER V6.22                                                      12/05/2013  00:54:40  PAGE 45


  C:4146H         SYMBOL        L?0373
  C:414CH         SYMBOL        L?0374
  -------         PROC          L?0372
  -------         ENDPROC       L?0372
  C:4146H         SYMBOL        L?0373
  C:414CH         SYMBOL        L?0374
  -------         PROC          _DELAYMS
  D:0010H         SYMBOL        value
  C:4150H         LINE#         2495
  C:4154H         LINE#         2496
  C:4154H         LINE#         2497
  C:415AH         LINE#         2498
  C:415AH         LINE#         2499
  C:4161H         LINE#         2500
  C:4169H         LINE#         2501
  C:416BH         LINE#         2502
  -------         ENDPROC       _DELAYMS
  -------         PROC          _DELAYUS
  D:0006H         SYMBOL        value1
  C:43A3H         LINE#         2507
  C:43A3H         LINE#         2508
  C:43A3H         LINE#         2509
  C:43A7H         LINE#         2510
  C:43AEH         LINE#         2511
  -------         ENDPROC       _DELAYUS
  -------         ENDMOD        LCD_DRIVE

  -------         MODULE        TOUCH
  C:0000H         SYMBOL        _ICE_DUMMY_
  D:0090H         PUBLIC        P1
  D:00B0H         PUBLIC        P3
  D:00A8H         PUBLIC        IE
  C:433EH         PUBLIC        _delay
  C:386BH         PUBLIC        _LCD_SetPos
  B:00B0H.7       PUBLIC        CS
  D:00B8H         PUBLIC        IP
  B:00B0H.6       PUBLIC        DCLK
  D:0024H         PUBLIC        coordinate
  D:0098H         PUBLIC        SCON
  C:430DH         PUBLIC        Read_7843
  D:0088H         PUBLIC        TCON
  C:3F51H         PUBLIC        pix_filter
  B:00B0H.4       PUBLIC        DOUT
  C:42EEH         PUBLIC        _Write_7843
  B:00B0H.5       PUBLIC        DIN
  C:42ACH         PUBLIC        AD7843
  C:40EBH         PUBLIC        _drawpoint
  D:0028H         PUBLIC        lx
  D:002AH         PUBLIC        ly
  D:00C8H         PUBLIC        T2CON
  C:43BBH         PUBLIC        start_7843
  B:00B0H.3       PUBLIC        Penirq
  C:3D32H         PUBLIC        Getpix
  D:00D0H         PUBLIC        PSW
  -------         PROC          _DRAWPOINT
  D:0005H         SYMBOL        x
  D:0082H         SYMBOL        y
BL51 BANKED LINKER/LOCATER V6.22                                                      12/05/2013  00:54:40  PAGE 46


  D:0008H         SYMBOL        color
  C:40EBH         LINE#         10
  C:40F5H         LINE#         11
  C:40F5H         LINE#         12
  C:4110H         LINE#         13
  C:4117H         LINE#         14
  C:411EH         LINE#         15
  C:4125H         LINE#         16
  -------         ENDPROC       _DRAWPOINT
  -------         PROC          _LCD_SETPOS
  D:000AH         SYMBOL        x0
  D:000CH         SYMBOL        x1
  D:000EH         SYMBOL        y0
  D:0010H         SYMBOL        y1
  C:386BH         LINE#         22
  C:3877H         LINE#         23
  C:3877H         LINE#         24
  C:3882H         LINE#         25
  C:388DH         LINE#         26
  C:3898H         LINE#         27
  C:38A3H         LINE#         29
  C:38ADH         LINE#         30
  C:38ADH         LINE#         31
  C:38B8H         LINE#         32
  C:38BEH         LINE#         33
  C:38BEH         LINE#         34
  C:38C9H         LINE#         35
  C:38C9H         LINE#         36
  C:38D5H         LINE#         37
  C:38E0H         LINE#         38
  C:38ECH         LINE#         39
  C:38F7H         LINE#         40
  C:3903H         LINE#         41
  C:390EH         LINE#         42
  C:391AH         LINE#         43
  C:3920H         LINE#         44
  C:3920H         LINE#         45
  C:3922H         LINE#         46
  C:392AH         LINE#         47
  C:392AH         LINE#         48
  C:3936H         LINE#         49
  C:3941H         LINE#         50
  C:394DH         LINE#         51
  C:3958H         LINE#         52
  C:3964H         LINE#         53
  C:396FH         LINE#         54
  C:397BH         LINE#         55
  C:3986H         LINE#         56
  C:3988H         LINE#         57
  C:398BH         LINE#         58
  C:3997H         LINE#         59
  C:3997H         LINE#         60
  C:399DH         LINE#         61
  C:39A5H         LINE#         62
  C:39ACH         LINE#         64
  C:39B3H         LINE#         65
  C:39BBH         LINE#         66
BL51 BANKED LINKER/LOCATER V6.22                                                      12/05/2013  00:54:40  PAGE 47


  C:39C2H         LINE#         68
  C:39C4H         LINE#         69
  C:39C6H         LINE#         70
  C:39D2H         LINE#         71
  C:39D2H         LINE#         72
  C:39D8H         LINE#         73
  C:39E0H         LINE#         74
  C:39E7H         LINE#         76
  C:39EEH         LINE#         77
  C:39F6H         LINE#         78
  C:39FDH         LINE#         80
  C:39FFH         LINE#         81
  C:3A01H         LINE#         83
  C:3A01H         LINE#         84
  C:3A0CH         LINE#         85
  C:3A17H         LINE#         86
  C:3A1EH         LINE#         87
  C:3A1EH         LINE#         89
  -------         ENDPROC       _LCD_SETPOS
  C:432FH         SYMBOL        L?0050
  C:4338H         SYMBOL        L?0051
  C:433AH         SYMBOL        L?0052
  -------         PROC          L?0049
  -------         ENDPROC       L?0049
  C:432FH         SYMBOL        L?0050
  C:4338H         SYMBOL        L?0051
  C:433AH         SYMBOL        L?0052
  -------         PROC          _DELAY
  D:0006H         SYMBOL        i
  C:433EH         LINE#         108
  C:433EH         LINE#         109
  C:433EH         LINE#         110
  C:4348H         LINE#         111
  -------         ENDPROC       _DELAY
  -------         PROC          START_7843
  C:43BBH         LINE#         116
  C:43BBH         LINE#         117
  C:43BBH         LINE#         118
  C:43BDH         LINE#         119
  C:43BFH         LINE#         120
  C:43C1H         LINE#         121
  C:43C3H         LINE#         122
  C:43C5H         LINE#         123
  -------         ENDPROC       START_7843
  -------         PROC          _WRITE_7843
  D:0005H         SYMBOL        temp
  -------         DO            
  D:0003H         SYMBOL        i
  -------         ENDDO         
  C:42EEH         LINE#         129
  C:42F0H         LINE#         130
  C:42F0H         LINE#         131
  C:42F2H         LINE#         133
  C:42F2H         LINE#         134
  C:42F2H         LINE#         135
  C:42FCH         LINE#         136
  C:42FFH         LINE#         137
BL51 BANKED LINKER/LOCATER V6.22                                                      12/05/2013  00:54:40  PAGE 48


  C:4304H         LINE#         138
  C:4308H         LINE#         139
  C:430CH         LINE#         140
  -------         ENDPROC       _WRITE_7843
  -------         PROC          READ_7843
  -------         DO            
  D:0005H         SYMBOL        i
  D:0002H         SYMBOL        temp
  -------         ENDDO         
  C:430DH         LINE#         146
  C:430DH         LINE#         147
  C:430DH         LINE#         148
  C:430FH         LINE#         149
  C:4311H         LINE#         151
  C:4311H         LINE#         152
  C:4311H         LINE#         153
  C:4318H         LINE#         154
  C:4318H         LINE#         155
  C:431BH         LINE#         156
  C:4323H         LINE#         157
  C:4327H         LINE#         158
  C:432BH         LINE#         159
  -------         ENDPROC       READ_7843
  -------         PROC          AD7843
  -------         DO            
  D:0011H         SYMBOL        pix
  -------         ENDDO         
  C:42ACH         LINE#         165
  C:42ACH         LINE#         166
  C:42ACH         LINE#         168
  C:42AEH         LINE#         170
  C:42B0H         LINE#         171
  C:42B0H         LINE#         172
  C:42B3H         LINE#         173
  C:42BAH         LINE#         175
  C:42BCH         LINE#         176
  C:42BCH         LINE#         177
  C:42BFH         LINE#         178
  C:42C6H         LINE#         180
  C:42C8H         LINE#         181
  C:42CEH         LINE#         182
  -------         ENDPROC       AD7843
  -------         PROC          PIX_FILTER
  D:0011H         SYMBOL        pix1
  D:0015H         SYMBOL        pix2
  -------         DO            
  D:0005H         SYMBOL        flag
  D:0006H         SYMBOL        x
  D:0002H         SYMBOL        y
  -------         ENDDO         
  C:3F51H         LINE#         188
  C:3F51H         LINE#         189
  C:3F51H         LINE#         190
  C:3F53H         LINE#         191
  C:3F75H         LINE#         192
  C:3F97H         LINE#         193
  C:3FADH         LINE#         194
BL51 BANKED LINKER/LOCATER V6.22                                                      12/05/2013  00:54:40  PAGE 49


  C:3FADH         LINE#         195
  C:3FAFH         LINE#         196
  C:3FC0H         LINE#         197
  C:3FD1H         LINE#         198
  C:3FD1H         LINE#         199
  C:3FD3H         LINE#         200
  -------         ENDPROC       PIX_FILTER
  -------         PROC          GETPIX
  -------         DO            
  D:0008H         SYMBOL        flag
  D:0009H         SYMBOL        pix1
  D:000DH         SYMBOL        pix2
  -------         ENDDO         
  C:3D32H         LINE#         205
  C:3D32H         LINE#         206
  C:3D32H         LINE#         207
  C:3D35H         LINE#         211
  C:3D3BH         LINE#         212
  C:3D3BH         LINE#         213
  C:3D4BH         LINE#         214
  C:3D5BH         LINE#         216
  C:3D89H         LINE#         217
  C:3D89H         LINE#         218
  C:3D9FH         LINE#         219
  C:3D9FH         LINE#         220
  C:3DC9H         LINE#         221
  C:3DF3H         LINE#         222
  C:3DF6H         LINE#         223
  C:3DF6H         LINE#         224
  C:3DF6H         LINE#         225
  C:3DF6H         LINE#         227
  C:3DF8H         LINE#         229
  -------         ENDPROC       GETPIX
  -------         ENDMOD        TOUCH

  -------         MODULE        ?C?FPMUL
  C:2F3BH         PUBLIC        ?C?FPMUL
  -------         ENDMOD        ?C?FPMUL

  -------         MODULE        ?C?FPDIV
  C:3044H         PUBLIC        ?C?FPDIV
  -------         ENDMOD        ?C?FPDIV

  -------         MODULE        ?C?FCAST
  C:30EBH         PUBLIC        ?C?FCASTC
  C:30E6H         PUBLIC        ?C?FCASTI
  C:30E1H         PUBLIC        ?C?FCASTL
  -------         ENDMOD        ?C?FCAST

  -------         MODULE        ?C?CASTF
  C:311FH         PUBLIC        ?C?CASTF
  -------         ENDMOD        ?C?CASTF

  -------         MODULE        ?C?COPY
  C:3270H         PUBLIC        ?C?COPY
  -------         ENDMOD        ?C?COPY

BL51 BANKED LINKER/LOCATER V6.22                                                      12/05/2013  00:54:40  PAGE 50


  -------         MODULE        ?C?LNEG
  C:3296H         PUBLIC        ?C?LNEG
  -------         ENDMOD        ?C?LNEG

*** WARNING L16: UNCALLED SEGMENT, IGNORED FOR OVERLAY PROCESS
    SEGMENT: ?PR?START_7843?TOUCH

Program Size: data=51.0 xdata=0 code=17359
LINK/LOCATE RUN COMPLETE.  1 WARNING(S),  0 ERROR(S)
